:080000000C9470000C94000048
:100008000C9400000C9400000C9400000C94000068
:100018000C9400000C9400000C9400000C94000058
:100028000C9400000C9400000C9400000C94000048
:100038000C9400000C9400000C94D2000C94000066
:100048000C949F000C9400000C9400000C94000089
:100058000C9400000C9400000C9400000C94000018
:100068001027E80364000A000100001000011000D6
:100078000100000000000A0000000000000000006D
:100088000000000000000000000000000000000068
:100098000000000000000000000000000000000058
:1000A8000000000000000000000000000000000048
:1000B800000000000A0A0A0A0A0A0A0A0A0A0A0AC0
:1000C8000A0A0A0A020002007A00020004007C0000
:1000D800010007037E000000F894EE27EFBBF1E073
:1000E800F5BFE5BF8DE0A2E0BB27ED938A95E9F760
:1000F80080E098E0A0E0B1E0ED930197E9F7ECEC3F
:10010800F0E085919591009761F0A591B5910590E2
:100118001590BF01F00105900D920197E1F7FB01E1
:10012800F0CFE8E0EEBBEFEFEDBFE8E0EEBFC0E0F8
:10013800D3E00C94E603AA93EA93FA93EFB7EA9311
:100148001A930A931091C0000091C600E12FEC7138
:10015800E9F4E0912404EF5FE0932404E150F0E037
:10016800E55FFB4F0083A0912404A93119F4E0E076
:10017800E0932404A0912604AF5FA0932604A9313C
:1001880029F4E0E0E0932604689437F8099119917E
:10019800E991EFBFF991E991A99118950A921A92FC
:1001A8006A937A938A939A93AA93BA93EA93FA935F
:1001B800EFB7EA93E0915503F09156033196E09337
:1001C8005503F09356030E94B230E1E5F1E00E9436
:1001D800FE3D0E2E0E94B230E3EAF2E00E94FE3DA0
:1001E800E02909F432C2A0915303B0915403E5E029
:1001F800F0E00E94223E0E2EA0912903EEE00E941C
:10020800F43DE02121F0E0912903EF5F03C025FCD4
:1002180003C0E0E0E0932903A0912903AE3011F474
:10022800689425F8A0913203A13029F4F79B02C005
:10023800F79801C0F79AE1E02E260E94B7300E9495
:10024800C030E093EB03F093EC036093ED037093FD
:10025800EE030E94C730AFECB3E00E94CC300E949E
:10026800D330ABEFB3E00E94CC300E94D8300E946C
:10027800E1300E94253DE093CF03F093D0036093D3
:10028800D1037093D203A091FB03B091FC0380913A
:10029800FD039091FE03E0E0F0E060E772E40E9465
:1002A800253DE093FB03F093FC036093FD037093FB
:1002B800FE030E94E6300E94EB300E2E0E94F030C2
:1002C8000E94EB30E02161F1E091FB03F091FC0327
:1002D8006091FD037091FE030E94D8300E94253D75
:1002E800E093F703F093F8036093F9037093FA032C
:1002F8000E94F530A7E6B3E00E94FE30A091F70314
:10030800B091F8038091F9039091FA030E94C030EC
:10031800E093D703F093D8036093D9037093DA037B
:100328000E9403310E940C310E9415310E94873CC3
:10033800E093DF03F093E0036093E1037093E2033B
:100348000E9403310E941E310E948A3D0E2E0E9497
:100358002331E8EEFDEF0E941C3EE021D1F00E941F
:1003680003310E940C31A0910304B09104048091E0
:100378000504909106040E942831E0930304F09349
:1003880004046093050470930604A5E7B3E00E9493
:10039800FE300E9403310E940C310E942D310E94D0
:1003A800873CE0930704F093080460930904709372
:1003B8000A040E9436310E943F310E942831A7EB7F
:1003C800B3E00E94163C0E94103F0E943631AAE01A
:1003D800B0E080E090E00E94503E0E942D310E94E3
:1003E8004B3C0E946A3D70F0E0E0E0930704E09324
:1003F8000804E0930904E0930A040E9452313196FC
:100408000E945731E091BB03F091BC036091BD039A
:100418007091BE030E9403310E94D73CDF01CB01DB
:100428000E94C030E093EF03F093F0036093F10370
:100438007093F2030E945C310E94873C0E946531F0
:10044800E0910E03F0E00E946E310E94CC3D0E94C4
:100458007731A9E8B3E00E9486310E94B7300E9444
:10046800703F3CF5A091EF03B091F0038091F10348
:100478009091F2030E948B317F936F93FF93EF93D8
:10048800A091EB03B091EC038091ED039091EE0302
:100498000E948B31AF91BF918F919F910E94253D12
:1004A800E093E703F093E8036093E9037093EA03AA
:1004B80009C0E0E0E093E703E093E803E093E90391
:1004C800E093EA03A091EA03AA238AF40E949231F6
:1004D8000E949B3118F40E94A23108C00E94A931E1
:1004E8000E94E13BA1E9B3E00E94863114C00E945A
:1004F8009231E0E0F0EC69E774E40E946A3D09F0AB
:1005080008F403C00E94A23106C00E94A931A1E9E3
:10051800B3E00E9486310E94B2310E94BB310E9432
:10052800873C0E94C431E091CF03F091D0036091E1
:10053800D1037091D2030E94CD310E946A3D68F5C3
:10054800E091D703F091D8036091D9037091DA0351
:100558000E94CD310E94873CE093D303F093D403EB
:100568006093D5037093D6030E94CD310E94D63193
:100578000E94803CDF01CB010E94F5300E94253D9E
:10058800A0E0B0E081E695E40E94D73CA5E8B3E09E
:100598000E948631689424F802C0E0E12E260E9469
:1005A800B2310E94DF310E94873CE093DB03F09375
:1005B800DC036093DD037093DE030E94DF31E0E02B
:1005C800F0E060E87FE30E946A3D09F008F412C099
:1005D800E093DB03E093DC03E093DD03E093DE03C9
:1005E8000E94E831EF5FFF4F6F4F7F4F0E94F1315C
:1005F8000E94FA310E940032A034E2E4BE07EFE024
:100608008E07E0E09E0778F0E0E0E0937703E09360
:100618007803E0937903E0937A03AFE5B0E00E94B2
:100628001E310E94453F0E94BB310E940932A7E556
:10063800B3E00E94FE30A0912703AC3308F4F2988F
:10064800A0912703AC3309F4F29A0E94B230A33A7E
:10065800E2E0BE0709F08DC0A09126030E940D328A
:100668000E9412320E941E310E94283E0E941B32B4
:10067800E02191F0E0912703EF5FE0932703E091F9
:100688002603F0E03296A0912703B0E0EA17FB07B3
:1006980019F4ECE3E0932703E0E0E0935503E093DB
:1006A8005603D394A0910F03A13028F4E0910F03CF
:1006B800EF5FE0930F030E942232E8E5F2E00E9428
:1006C8001C3E0E2E0E942732E02199F0E0916B0328
:1006D800F0916C033196E0936B03F0936C030E94E6
:1006E80022320E942C32EA1BFB0BE0937103F09339
:1006F8007203ECE3ED1589F4DD24C394EC1569F479
:10070800CC24E0910003EF5FE0930003A091000385
:10071800A43119F4E0E0E0930003A0912E03A13086
:10072800D0F0E0911203EF5FE0931203A09112035F
:10073800A23088F0E0911103EF5FE0931103E0E04D
:10074800E0931203E0912E03A0911103EA1718F425
:10075800E0E0E0931103E0912E03E03019F4E0E0CB
:10076800E0931103A0912E03A23019F4E1E0E09385
:100778001103E991EFBFF991E991B991A991999183
:10078800899179916991199009901895AA93E881AE
:10079800E066E0937C0085E28A95F1F7E0917A00C3
:1007A800E064E0937A00E0917A00E071E1F3E0918F
:1007B8007A00E061E0937A00E0917800F0917900A6
:1007C80021960895EF9763978CE4A6E0B0E0E0E8FF
:1007D800F0E00E94853FFF2411E001E0E0E8E093AB
:1007E8006100E0E0E0936100EFE0E4B9E1E0E5B941
:1007F800E0E0E7B9E4E0E8B9EAEFEAB9E7EEEBB937
:10080800E0E0E4BDE3E0E5BDE0E0E6BDE7BDE8BD6E
:10081800E0938000E0938100E0938500E0938400FA
:10082800E0938700E0938600E0938900E0938800D6
:10083800E0938B00E0938A00E093B600E1EAE0934E
:10084800B000E2E0E093B100E0E0E093B200E093B2
:10085800B300E093B400E1E0E0936E00E0E0E093E1
:100868006F00E0937000E0936900EDBBE0936800CF
:10087800E093C000E8E9E093C100E6E0E093C2003D
:10088800E0E0E093C500E7E4E093C400E0E8E0BFFF
:10089800E0E0E0937F00E0937E00E0E6E0937C00F8
:1008A800E6E2E0937A00E0E0E0937B00ECBDE093C1
:1008B800BC0078945F9A0E9431320E9435320E94BF
:1008C8003B320E9442320E944F320E943132EAE0AB
:1008D8006E16B8F5ABE3B0E00E945C32A6E2B0E079
:1008E800E0E00E94553FA7E2B0E00E94553FA6E332
:1008F800B0E00E94553FA7E3B0E00E94553FA8E34F
:10090800B0E00E94553FA1E5B0E0E8EEF3E00E94B8
:100918004D3FA3E5B0E00E945C32A5E5B0E00E943F
:100928005C32A7E5B0E00E945C32A9E5B0E00E9425
:100938005C32ABE5B0E00E945C32ADE5B0E00E940D
:100948005C32EAE09E1650F4A1E4B0E00E945C320A
:10095800A9E4B0E00E945C32689426F8EAE0BE168A
:1009680018F4689430F827F8689433F8E9E1E093CC
:1009780016030E946132E8ECF0E00E946832E0ED74
:10098800F7E00E946D32E8ECF0E0E0937F03F0932B
:100998008003A0E0B0E00E94393FE0931703A1E094
:1009A800B0E00E94393FE0931803A2E0B0E00E9453
:1009B800393FE0931903A3E0B0E00E94393FE09388
:1009C8001B03A4E0B0E00E94393FECA7A5E0B0E02B
:1009D8000E94393FEDA7A6E0B0E00E94393FEEA79C
:1009E800A7E0B0E00E94393FE0931C03A8E0B0E024
:1009F8000E94393FE0931D03F798F198AAE0B0E010
:100A08000E94393FE0932603A9E3B0E00E94353FF6
:100A18000E947232A2E1B0E00E94393FE8A7A3E148
:100A2800B0E00E94393FE9A7A4E1B0E00E94393F55
:100A3800EAA7ABE0B0E00E94393FECA3ACE0B0E03D
:100A48000E94393FEDA3ADE0B0E00E94393FEEA32C
:100A5800ADE3B0E00E94353FEB8BFC8BAEE0B0E03D
:100A68000E94393FE0933303AFE0B0E00E94393F82
:100A7800E0933503A0E1B0E00E94393FE0933403EE
:100A8800AFE5B0E00E94313F0E94F131ABE3B0E046
:100A98000E94353FABECB3E00E9477320E94D6311A
:100AA800A7E5B3E00E94FE300E94BB310E947E326F
:100AB8000E94C431A1E1B0E00E94393FF0E0EB8729
:100AC800FC87AFE3B0E00E94353FEF8BF88FAFE4CF
:100AD800B0E00E94353FED87FE87A1E4B0E00E94B8
:100AE800353FAFEDB3E00E947732A9E4B0E00E9451
:100AF800353FAFEFB3E00E9477320E945C310E942D
:100B08007E320E946531A3E4B0E00E94353F0E9426
:100B18008232A7E4B0E00E94353F0E94CC3D0E949B
:100B28008732A5E1B0E00E94393F0E94803F23F858
:100B3800A5E4B0E00E94353F0E949032A6E1B0E003
:100B48000E94393FE0930603A7E1B0E00E94393FD5
:100B5800E0930803A8E1B0E00E94393FE09309035D
:100B6800A9E1B0E00E94393FE0930A03AAE1B0E0AE
:100B78000E94393FE0930B03ABE1B0E00E94393F9C
:100B8800E0930C03ACE1B0E00E94393FE0932A0304
:100B9800ADE1B0E00E94393FE0932B03AEE1B0E055
:100BA8000E94393FE0932C03AFE1B0E00E94393F47
:100BB800E0932D03A0E2B0E00E94393FE0932E03BA
:100BC800A1E2B0E00E94393FE0932F03A2E2B0E037
:100BD8000E94393FE0933003A3E2B0E00E94393F1E
:100BE800E0933103ABE4B0E00E94353F0E945731F7
:100BF800A4E2B0E00E94393FE0930E03A5E2B0E022
:100C08000E94393F0E94803F36F8A8E2B0E00E9477
:100C1800393FE0931003A9E2B0E00E94393FEF8F1B
:100C2800ADE4B0E00E94353FEF87F88BAAE2B0E070
:100C38000E94393FE0934103ABE2B0E00E94393FA4
:100C4800E0934203ACE2B0E00E94393FE0934303F3
:100C5800ADE2B0E00E94393FE0931E03AEE2B0E09F
:100C68000E94393FE0932003A9E0B0E00E94393F99
:100C7800E0932103AFE2B0E00E94393FE093220302
:100C8800A0E3B0E00E94393FE0932303A1E3B0E082
:100C98000E94393FE0931503A2E3B0E00E94393F78
:100CA800E0934A03A3E3B0E00E94393FE0934B038B
:100CB800A4E3B0E00E94393FE0934C03A5E3B0E021
:100CC8000E94393FE0934E030E949532E0937503EA
:100CD800F09376030E949532A3E0B4E00E94773245
:100CE80036FE0BC0A6E2B0E00E94393FCE2EA7E246
:100CF800B0E00E94393FE0930003E1E0E0933F0356
:100D0800A0910203AE3128F4E0910203EF5FE09373
:100D18000203A0910203AE3189F4E0E0E0933803C6
:100D2800E0939903E0939A03EBE0F0E00E949A3293
:100D3800E8EB0E949F32E4E1E0930203EF8DE0309C
:100D480041F5A0910B04ECE30E94D63D0E2EA09134
:100D58000C04E7E00E94D63D0E22A0912404EBE0AB
:100D68000E94D63DE02169F0E0910D04E09337033D
:100D7800E0910E04E09338030E94A532E0E0E0938E
:100D88000203A0912404AC3020F00E94B3320E94E8
:100D9800BF32AF8DA130D1F4A0910B04E8E20E94DC
:100DA800D63D0E2EA0912404E8E00E94D63DE02115
:100DB80029F00E94A532E0E0E0930203A091240408
:100DC800AC3020F00E94B3320E94BF32AF8DA33006
:100DD80009F079C0A0910B04ECE60E94D63D0E2ED6
:100DE800A0910C04EBE00E94D63D0E22A0912404B1
:100DF800EFE00E94D63DE02109F441C0E0910E04E5
:100E0800E0933703E0910F04E0933803E091100476
:100E1800F0E00E94CB32F0919903E0E00E94CB32DF
:100E2800E0911104F0E0A0919903B0919A03EA0FC0
:100E3800FB1F0E94CB32E0911204E0934803E0913B
:100E48001504E0934703E0911604F0E00E949A32FB
:100E5800E0911704E0933903E0911304F0E0E09384
:100E68009B03F0939C03E0911404F0E0E0939D034E
:100E7800F0939E03E0E0E0932404E0930203A09142
:100E88002404A03100F1E0E0E0930B04E0930C04AB
:100E9800E0930D04E0930E04E0930F04E093100434
:100EA800E0931104E0931204E0931304E093140414
:100EB800E0931504EBE0E0931604E8EBE0931704E5
:100EC800E0E0E0932404E8EC5E1630F45394EEE19D
:100ED800E51511F4E1E04E2E0E94D032E7EAE093E6
:100EE8007A00A6E00E94D432EF83F887E7E2E09325
:100EF8007A000E94D0320E9435320E94C13D0E9481
:100F0800BD3DE987FA87E7E2E0937A000E94D03294
:100F18000E94DB323B97A0F1A0E00E94D432662702
:100F280077270E94E432A8EEB3E080E090E00E94C8
:100F38007B3EDF01CB010E94ED32662777270E94B6
:100F4800BD3E0E94E432ABEBB3E00E944D3C0E94F0
:100F5800103FE0910703EF5FE0930703E09106037A
:100F6800A0910703AE1750F00E94F232E093B3034A
:100F7800F093B4036093B5037093B603E894F3F861
:100F88000E94FB320E9435320E943B320E9402339B
:100F9800A2E00E94D432DF01E5E0F0E00E94803E4A
:100FA8008E2E0E94FB320E944F328AE48A95F1F716
:100FB8000E9442320E9402330E9409330E94FB328F
:100FC800E7EAE0937A00A5E0E1DBEF2FF0E0E98FB4
:100FD800FA8F0E94FB320E94DB32AE2E0E94FB3257
:100FE800A0914E03A13069F4E98DFA8DA98DBA8DCF
:100FF8000E94483EDF01E6EDF0E00E94803EE98F66
:10100800FA8FE0911003E03009F0A0C0E1E0E515A7
:10101800B1F50E9413335E9710F4E1E0EAA30E9451
:1010280013330E9418330E941333EAEFF0E00E9452
:101038001C3EE02111F0E2E0EAA30E941333AB3F2B
:10104800E0E0BE0710F0E3E0EAA3A98DBA8D5E9751
:1010580010F4E1E0E9A30E941E33A98DBA8DEAEFEE
:10106800F0E00E941C3EE02111F0E2E0E9A3A98D26
:10107800BA8DAB3FE0E0BE0710F0E3E0E9A30E94C1
:1010880013330E942133AAA10E942C3311F0E4E00B
:1010980009C00E9413330E943133AAA10E942C3345
:1010A80011F0E5E0EAA3A98DBA8D0E942133A9A128
:1010B8000E942C3311F0E4E009C0A98DBA8D0E947A
:1010C8003133A9A10E942C3311F0E5E0E9A3AAA1CC
:1010D8000E940D32AAA10E943C3369F0E98DFA8D75
:1010E8000E944133E8E2F0E0E98FFA8FAE81AC3537
:1010F80011F40E944633AAA10E944C33AAA1E5E04C
:101108000E94D63DE02911F00E944633A9A10E9411
:101118000D32A9A10E943C3369F0E8E2F0E0E98FC2
:10112800FA8FAAA10E940D32AAA10E943C3311F0A5
:101138000E944633A9A10E944C330E945133E029F2
:1011480021F0ECE3F0E0E98FFA8F03C0E0E0EAA3D6
:10115800E9A3A98DBA8DA73DE0E0BE0720F0E6ED32
:10116800F0E0E98FFA8F0E9456330E945C330E94A8
:10117800F43DE021E9F1E4E1ED8F6894F3F80E9491
:1011880066330E946C3319F0E1E0E0931403A12F59
:101198000E9475330E947A3321F0F398F49A12E092
:1011A8001CC0A12FE2E00E94D63D0E2E0E947A3389
:1011B80059F0F498F59AAEA5A13010F013E003C0E9
:1011C800F598F39A11E009C0A12F0E947D330E947F
:1011D8007A3319F0F598F39A11E0A62DE9E00E9408
:1011E800F93D0E2E0E946C3319F0E0E0E0931403F1
:1011F800E0914F03E09340030E941333D39708F420
:101208005DC00E9482330E948733E12F0E948E3393
:1012180020F0E8ECF0E00E944133A0914203A130B5
:1012280011F40E949E33E12F0E94A9330E94B93322
:10123800AC91A13008F441C00E94C0330E94C93368
:101248000E947B3F4CF40E94B9330E94D5330E9420
:10125800963D0E94DF3323C00E94E8330E94EA33A0
:10126800EF930E94E8330E94F333AF91EA2379F0B9
:101278000E94B9330E94D5330E949B3DA093A303DB
:10128800B093A4038093A5039093A60308C00E947B
:10129800E8330E94FC331CF00E9406340EC0A09173
:1012A800A303B091A4038091A5039091A6030E9483
:1012B80015340E94BD3E0E94413304C00E9446334B
:1012C8000E9406340E9466330E941A340E220E943D
:1012D8001F3401F10E9413330E946C3F10F4E4E1C3
:1012E800EB8FA09128030E940D320E942334E02145
:1012F80041F0E3E0E0933603E0E0E09328030E9446
:101308002934E0914F03E09328036894F0F821F81A
:10131800E894F4F8A0913003A130D9F50E942F3455
:101328000E2EA0914003E0E50E94F43D0E22A0910C
:101338002803E8EC0E94F43D0E9431340E22A0E01C
:10134800F4FCA1E00E94393429F0E0912803EF5F12
:10135800E09328030E941E33A98DBA8DE0E5F0E0E2
:101368000E941C3E0E22A0912803E0E00E94F93D55
:101378000E943134E02169F0E0912803E150E093C4
:1013880028030E943E340E94423419F0E3E00E9490
:1013980048340E9423340E944B34A09128030E94B1
:1013A8002C3321F0E0E0E093290306C0A091290343
:1013B800A23010F4E89425F8A0912803A13020F079
:1013C800E0912803F0E002C00E948233E0935303C7
:1013D800F09354030E948233309729F4E89421F85B
:1013E8006894F4F827C00E9454340E2E0E942F34BB
:1013F8000E22A09130030E942C331E2EA0912803A8
:101408000E940D320E9454340E22A0914003EFE452
:101418000E94F93D0E22A09130030E943934E1293F
:1014280049F0E0E0E09328030E944633E89422F86C
:10143800689421F8E09104030E941333F0E0EA175E
:10144800FB0720F4E0914F03E09304030E945B3410
:101458000E94403E0E22A09133030E942C331E2E80
:101468000E945B340E94383E0E22A09134030E94F1
:101478002C33E12961F0E0914F03E09304030E94CB
:101488003E340E946A3419F0E2E00E944834A09188
:101498002803A13080F0689422F80E948233A0913A
:1014A8002803B0E0AE17BF0728F0E0912803F0E06A
:1014B8000E94413302C0E89422F80E946E340E2242
:1014C800A0E031FCA1E00E942C3331F0689431F89F
:1014D8000E9482330E9468320E946E34E02161F1DA
:1014E8000E9484340E948C34A4F0A091AF03B09180
:1014F800B003EB89FC89EA1BFB0BA3E0B0E00E9478
:10150800763E0E949434AE1BBF0BA0938103B09328
:1015180082030E9484340E94703F2CF40E94993404
:1015280032970E946832A0918203AA232AF4E0E04D
:10153800E0938103E09382030E949E340E94763FE9
:1015480084F50E949E340E949B3D0E948C3474F066
:10155800AB89BC89E091AF03F091B003EA1BFB0BA8
:101568000E949434EA0FFB1F0E9468320E949E3446
:101578000E949B3DA230E0E0BE07E0E08E07E0E07D
:101588009E072CF00E94993431960E9468320E947E
:101598009434AB3FE0E0BE0724F0EAEFF0E00E94AD
:1015A80068320E9499340E941333AE17BF0710F4B3
:1015B800E89431F80E9499340E941333EA17FB0724
:1015C80020F40E9499340E9441330E94AB34A0E079
:1015D80032FCA1E00E94BD340E94423431F068948C
:1015E80032F80E94C2340E946D320E94AB340E94CD
:1015F8004234A1F10E94C734DF01CB01E0E0F0E002
:1016080060E070E40E946A3D09F008F414C00E948A
:10161800C734A0E0B0E080E890E40E94D73C0E9484
:10162800D6340E94D13D0E94213F0E942831A3E870
:10163800B3E00E9486310E94C7340E94663F2CF4B2
:101648000E94DB3435970E946D32A0918403AA234F
:101658002AF4E0E0E0938303E0938403EB85FC85C0
:101668000E94E0340E94E9340E948A3D0E2E0E94B6
:101678004234A9F10E94EE34DF01CB01E0E0F0E052
:1016880060E470E40E946A3D09F008F414C00E9406
:10169800EE34A0E0B0E080EA90E40E94D73CDF019D
:1016A800CB010E94DB340E94FD340E94873CA3E8F2
:1016B800B3E00E9486310E94EE340E94663F2CF40B
:1016C8000E94DB3435960E946D320E94D634A53CC8
:1016D800E9E0BE0724F0E4ECF9E00E946D320E94D4
:1016E800C234DF010E94DB340E941C3E0E2E0E9491
:1016F800423411F0E89432F80E94C234DF010E94AB
:10170800DB340E94223E0E2E0E94423421F00E94B9
:10171800D6340E9402350E9407350E94403E0E2EA4
:10172800A0E034FCA1E00E942C3331F0689434F836
:101738000E94C2340E940E350E9407350E94763FEF
:101748005CF50E9413350E948C349CF0E0911803DC
:10175800F0E0A091AB03B091AC03AE1BBF0BE3E08C
:10176800F0E00E941C35AE1BBF0BA0938B03B09317
:101778008C030E9413350E94703F2CF40E9423357D
:1017880032970E940E35A0918C03AA232AF4E0E038
:10179800E0938B03E0938C030E9407350E947B3F04
:1017A8008CF50E942835A430E0E0BE07E0E08E0703
:1017B800E0E09E078CF0A0911803BB27E091AB03F3
:1017C800F091AC03AE1BBF0BE2E0F0E00E941C35C9
:1017D800EA0FFB1F0E940E350E9428350E94703FB9
:1017E8002CF40E94233532960E940E35A0918B036B
:1017F800B0918C03A53CE9E0BE0724F0E4ECF9E0E5
:101808000E940E350E94C234DF010E942335AE17B4
:10181800BF0710F4E89434F80E94C234DF010E9434
:101828002335EA17FB0730F4A0918B03B0918C03A2
:101838000E940235E09113030E941333F0E0EA1787
:10184800FB0720F4E0914F03E0931303E0911303A7
:10185800F0E035970E9413330E941C3E6E2F0E2E27
:10186800A0E031FCA1E00E9439341E2E062EA0E033
:1018780032FCA1E00E9439341E2A062EA0E034FC76
:10188800A1E00E943934E12961F0E0914F03E0932F
:1018980013030E943E340E94423419F0E2E00E9491
:1018A8004834A0913603A13078F00E944633A091C5
:1018B8003603A13021F4EAE0F0E00E944133E091E0
:1018C8003603E150E09336030E941E33A0913003A3
:1018D8000E942C331E2EA98DBA8DE0E5F0E00E94FF
:1018E800223E0E2EA0913003E1E00E94D63D0E94D8
:1018F8003134E0211E2A0E941E33A0913003E1E01A
:101908000E94D63D0E220E946A34E129E9F0E0E007
:10191800E0930503A0912803A13018F0E2E0E093DA
:101928003603E0E0E0932803E98DFA8DF2970E94F0
:10193800E934A6EFB8E28CE99FE30E94D73CDE01C8
:1019480059960E94FE3003C0E0E0E98FEA8F0E94BA
:101958008233E98BFA8B0E9438350E2EA0912B0327
:101968000E94393411F0299A01C029980E9438350B
:101978000E2EA0914103E2E00E94D63DE02111F035
:10198800EFEF01C0E0E0E09344030E9466330E9459
:101998001A34E02119F0E98DE0934D03A0914D032D
:1019A800A13068F0E0914D03F0E0E98FFA8F0E94D2
:1019B80013330E946C3F18F4E0E0E0934D03A82D28
:1019C800E4E60E94F43D6E2F0E2E0E943B350E2257
:1019D800AE81EDE50E94DB3D0E9442351E2E062EAB
:1019E8000E943B350E220E941A34E0211E2A0E94D2
:1019F8002C320E9422320E94FE3D0E9449350E94EC
:101A08002732E021E12941F1E0915703F091580391
:101A1800ABE3B0E00E9451350E9457350E945C311B
:101A28000E9409320E9464350E946935EC2DA6E2B5
:101A3800B0E00E946D35E0910003A7E2B0E00E949B
:101A48006D350E9473350E9431325F98A8EEB3E07D
:101A58000E94D73B5F98FECFAB2D0E947C350E9439
:101A68001A34E02131F0E894F2F827F8E0E0E09346
:101A78003D030E9481350E941A34E02171F0E09103
:101A88003D03EF5FE0933D03A0913D03AA3029F4A5
:101A9800E0E0E0933D03E09332030E948135A0E04B
:101AA800F2FCA1E00E94BD340E941A34E021C1F189
:101AB800E4E1EC8F6894F2F8E0913203EF5FE09391
:101AC8003203A09132030E947D330E941F3419F023
:101AD800E1E0E0933203A09132030E944C330E946C
:101AE8001F3419F0E2E0E0933203A09132030E9420
:101AF8007D33A0912B030E94BD340E94423419F01B
:101B0800E1E0E0933203A09132030E944C33A0E05D
:101B1800F0FCA1E00E94393419F0E3E0E0933203CD
:101B2800E0913203E03031F4F7982A98E0E0E0934E
:101B380045031EC0A0913203A13031F42A98EFEF7B
:101B4800E0934503E0E014C0A0913203A23039F4D9
:101B5800F79A2A98EFEFE0934503E0E009C0A091D7
:101B68003203A33039F4F79A2A9AEFEFE09345034A
:101B7800E09346030E948A35E081E093B4000E9416
:101B88002F340E2E0E9438350E220E946A3429F115
:101B9800A0912A03A13009F45C9AE0910303EF5F56
:101BA800E0930303A0910303E5E00E94F93D0E2EA4
:101BB800E4E10E94F43DE02141F0E0910303E1708B
:101BC800AFEFEA02F001E093B400A0910303A03163
:101BD80018F0E0E0E093030325C05C98A0E030FC37
:101BE800A1E00E947533A09132030E942C33D1F0FA
:101BF800E0913C03EF5FE0933C03A0913C03A130EC
:101C080019F4EFEFE093B400A0913C03A33019F46A
:101C1800E0E0E093B400A0913C03A43019F4E0E0C4
:101C2800E0933C030E9490350E949735E1F0E091E3
:101C38001D03A0911F03AE1728F4E0911F03EE5F68
:101C4800E0931F03E0911D03A0911F03EA1728F4F6
:101C5800E0911F03E250E0931F03033621F4E09163
:101C68001D03E0931F030E949035EA17FB07E0F479
:101C7800E0911E03A0911F03AE1728F4E0911F0303
:101C8800EE5FE0931F03E0911E03A0911F03EA1784
:101C980028F4E0911F03E250E0931F03033621F478
:101CA800E0911E03E0931F03E0911F03E093B3004C
:101CB800EAE0E91518F4E894F1F826F80E94A0354E
:101CC800A0E026FCA1E00E94BD34A0E0F1FCA1E068
:101CD8000E94BD340E941A34E02139F16894F1F869
:101CE800E0910D03EF5FE0930D03E0E0E8A3A8A106
:101CF800A53088F40E94A635A081A13018F0E5E04F
:101D0800E8A305C0E0910D03EF5FE0930D03E8A1A0
:101D1800EF5FE8A3ECCFA0910D03A53018F0E0E049
:101D2800E0930D030E94A63500810E94A035A09182
:101D38002503EFEF0E94F43DE02121F0E091250317
:101D4800EF5F03C0E894F1F8E0E0E0932503A09189
:101D58002503A43109F087C1AE81E0E00E94EA3D85
:101D68000E2E0E941A34E02119F0EE81E150EE8324
:101D7800033610F403E677C101E0E0E0E0930D03D9
:101D8800E0911703A0E0B0E00E946D35E0911803E0
:101D9800A1E0B0E00E946D35E0911903A2E0B0E047
:101DA8000E946D35E0911B03A3E0B0E00E946D3501
:101DB800ECA5A4E0B0E00E946D35EDA5A5E0B0E08B
:101DC8000E946D35EEA5A6E0B0E00E946D35E09169
:101DD8001C03A7E0B0E00E946D35E0911D03A8E068
:101DE800B0E00E946D35E0912103A9E0B0E00E94C7
:101DF8006D35E0912603AAE0B0E00E946D350E949F
:101E0800ED32A9E3B0E00E945135E8A5A2E1B0E0C7
:101E18000E946D35E9A5A3E1B0E00E946D35EAA501
:101E2800A4E1B0E00E946D35ECA1ABE0B0E00E9407
:101E38006D35EDA1ACE0B0E00E946D35EEA1ADE0EE
:101E4800B0E00E946D35EB89FC89ADE3B0E00E94FB
:101E58005135E0913303AEE0B0E00E946D35E0917A
:101E68003503AFE0B0E00E946D35E0913403A0E1A6
:101E7800B0E00E946D35EB85A1E1B0E00E946D35C0
:101E8800EF89F88DAFE3B0E00E945135ED85FE850E
:101E9800AFE4B0E00E9451350E9457350E94AC353E
:101EA800A3E4B0E00E945135E0917B03F0917C03FC
:101EB800A7E4B0E00E945135E0E023FCE1E0A5E1B1
:101EC800B0E00E946D350E942C32A5E4B0E00E947B
:101ED8005135E0910603A6E1B0E00E946D35E0912E
:101EE8000803A7E1B0E00E946D35E0910903A8E17D
:101EF800B0E00E946D35E0910A03A9E1B0E00E94CC
:101F08006D35E0910B03AAE1B0E00E946D35E091D8
:101F18000C03ABE1B0E00E946D350E945C310E9479
:101F280009320E946435E0912A03ACE1B0E00E94D6
:101F38006D35E0912B03ADE1B0E00E946D35E09185
:101F48002C03AEE1B0E00E946D35E0912D03AFE1C6
:101F5800B0E00E946D35E0912E03A0E2B0E00E944F
:101F68006D35E0912F03A1E2B0E00E946D35E0915C
:101F78003003A2E2B0E00E946D35E0913103A3E2A4
:101F8800B0E00E946D350E946935E0910E03A4E22D
:101F9800B0E00E946D35E0E036FCE1E0A5E2B0E09B
:101FA8000E946D35E0911003A8E2B0E00E946D3503
:101FB800EF8DA9E2B0E00E946D35EF85F889ADE4B8
:101FC800B0E00E945135E0914103AAE2B0E00E94DE
:101FD8006D35E0914203ABE2B0E00E946D35E091CF
:101FE8004303ACE2B0E00E946D35E0911E03ADE220
:101FF800B0E00E946D35E0912003AEE2B0E00E94AF
:102008006D35E0912203AFE2B0E00E946D35E091BA
:102018002303A0E3B0E00E946D35E0911503A1E32E
:10202800B0E00E946D350E94FA31A1E0B0E00E9454
:10203800D73BE0914A03A2E3B0E00E946D35E091FE
:102048004B03A3E3B0E00E946D35E0914C03A4E399
:10205800B0E00E946D35E0914E03A5E3B0E00E9428
:10206800553FE1E04E2E0E94A035A0E0F1FCA1E032
:102078000E94BD34AE81E4E60E94E53D0E944235EF
:1020880051F06894F1F8EE81EF5FEE83AE81A436EB
:1020980011F4E0E0EE83EAE0E61510F4E894F0F8D5
:1020A8000E946633A0E0F0FCA1E00E94BD34AE813E
:1020B800E0E00E94E03D0E94423551F06894F0F85B
:1020C800EE81E150EE83AE81AF3F11F4E3E6EE839B
:1020D8000E9456330E94B135C1F00E94B735A9F469
:1020E800A0913A03A43119F4E7E0E0933A03E0E061
:1020F800E0933B03E894F3F8A0913A03A33028F067
:10210800E0913A03E150E0933A03AB2DEAE00E94F4
:10211800F43D0E2E0E94B135C1F00E94B735A9F4E6
:10212800A0913A03A43119F4E7E0E0933A03E0E020
:10213800E0933B03E894F2F8A0913A03A33028F027
:10214800E0913A03E150E0933A03AB2D0E947C35CD
:10215800AA2DEAE00E94F93DE02131F0E0E0E093A9
:102168003B03E4E1E0933A03EAE0EA1510F4E8946B
:10217800F3F80E9456330E945C330E94D63DE0215A
:1021880009F424C36894F3F8AE81A13049F4A0910E
:102198001703A13028F4E0911703EF5FE0931703CA
:1021A800AE81A23049F4A0911803AF3528F4E0912C
:1021B8001803EB5FE0931803AE81A33049F4A091B4
:1021C8001903A63928F4E0911903EF5F0E94C2357C
:1021D800AE81A43049F4A0911B03A83228F4E09101
:1021E8001B03EF5FE0931B03AE81A53031F4ACA570
:1021F800A43618F4ECA5EF5FECA7AE81A63031F455
:10220800ADA5A43618F4EDA5EF5FEDA7AE81A73014
:1022180031F4AEA5A43618F4EEA5EF5FEEA7AE81B3
:10222800A83049F4A0911C03AF3F28F4E0911C03A7
:10223800EF5FE0931C03AE81A93049F4A0914103FC
:10224800AF3F28F4E0914103EF5FE0934103AE8193
:10225800AA3049F4A0914203AF3F28F4E091420329
:10226800EF5FE0934203AE81AB3049F4A0914303A2
:10227800AF3F28F4E0914303EF5FE0934303AE815F
:10228800AC3049F4A0910E03A03328F4E0910E037A
:10229800E45FE0930E03AE81AD3069F4A091590379
:1022A800B0915A03A43CE9E0BE0728F40E94ED323D
:1022B80031960E947232AE81AE3031F4A8A5A436B0
:1022C80018F4E8A5EB5FE8A7AE81AF3031F4A9A513
:1022D800A43618F4E9A5EB5FE9A7AE81A03131F483
:1022E800AAA5A43618F4EAA5EB5FEAA7AE81A13146
:1022F80031F4ACA1A83C18F4ECA1EB5FECA3AE81DF
:10230800A23131F4ADA1A83C18F4EDA1EB5FEDA327
:10231800AE81A33131F4AEA1A83C18F4EEA1EB5F75
:10232800EEA3AE81A43169F4A0916903B0916A0368
:10233800A835E2E0BE0728F40E942C327E960E945F
:102348009032AE81A53189F4A0910E03EAE0EA9FAC
:10235800F001EA5BFF4FAB89BC89AE17BF0728F4D1
:10236800EB89FC893196EB8BFC8BAE81A63149F465
:10237800A0913303A13028F4E0913303EF5FE09399
:102388003303AE81A73149F4A0913503A23328F471
:10239800E0913503EF5FE0933503AE81A83149F44E
:1023A800A0913403A13028F4E0913403EF5FE09367
:1023B8003403AE81A931E1F4AB85BC85E9E1F0E0F5
:1023C8000E94D5350E942C3329F0EB85FC85319687
:1023D800EB87FC87AB85BC85E2E3F0E00E94D5354E
:1023E8000E94393429F0EB85FC853196EB87FC8710
:1023F800AE81AA3159F40E94DC35A03BE4E0BE0767
:1024080028F40E94AC3531960E94E135AE81AB319B
:1024180091F40E946E31A73EE3E0BE07E0E08E072C
:10242800E0E09E0740F40E943631EF5FFF4F6F4FA8
:102438007F4F0E948732AE81AC3161F4A0E023FC6B
:10244800A1E0A13038F4E0E023FCE1E0EF5F0E9476
:10245800803F23F8AE81AD3169F40E94E630AE3D8D
:10246800E3E0BE0738F40E94C7303A96E093610370
:10247800F0936203AE81AE3169F40E94F030A83562
:10248800E2E0BE0738F40E94D3303A96E0936D0339
:10249800F0936E03AE81AF3149F4A0910603AA30E0
:1024A80028F4E0910603EF5FE0930603AE81A032C3
:1024B80049F4A0910803AC3028F4E0910803EF5FD9
:1024C800E0930803AE81A13249F4A0910903AC302E
:1024D80028F4E0910903EF5FE0930903AE81A2328B
:1024E80049F4A0910A03AC3028F4E0910A03EF5FA5
:1024F800E0930A03AE81A33249F4A0910B03AC30F8
:1025080028F4E0910B03EF5FE0930B03AE81A43254
:1025180049F4A0910C03AC3028F4E0910C03EF5F70
:10252800E0930C03AE81A53249F4A0912A03A130AF
:1025380028F4E0912A03EF5FE0932A03AE81A632E4
:1025480049F4A0912B03A13028F4E0912B03EF5F0D
:10255800E0932B03AE81A73249F4A0912C03A2305B
:1025680028F4E0912C03EF5FE0932C03AE81A832AE
:1025780049F4A0912D03A13028F4E0912D03EF5FD9
:10258800E0932D03AE81A93249F4A0912E03A23025
:1025980028F4E0912E03EF5FE0932E03AE81AA3278
:1025A80049F4A0912F03A33028F4E0912F03EF5FA3
:1025B800E0932F03AE81AB3249F4A0913003A130F0
:1025C80028F4E0913003EF5FE0933003AE81AC3242
:1025D80049F4A0913103A13028F4E0913103EF5F71
:1025E800E0933103AE81AD3291F40E940032AF39ED
:1025F800E6E8BE07E1E08E07E0E09E0740F40E94AF
:10260800E831E65FFF4F6F4F7F4F0E94F131AE8197
:10261800AE3259F40E94FA35A031E7E2BE0728F439
:102628000E9452313A960E945731AE81AF3261F41E
:10263800A0E036FCA1E0A13038F4E0E036FCE1E0AF
:10264800EF5F0E94803F36F8AE81A03349F4A09135
:102658001003A13028F4E0911003EF5FE09310031A
:10266800AE81A13331F4AF8DA33018F4EF8DEF5F55
:10267800EF8FAE81A23359F4AF85B889A632E2E074
:10268800BE0728F4EF85F8893196EF87F88BAE817D
:10269800A33349F4A0911503A43628F4E091150357
:1026A800EF5FE0931503AE81A43341F40E94FF3538
:1026B800A23820F40E940636EF5FEC93AE81A53372
:1026C80049F4A0914E03A13028F4E0914E03EF5F46
:1026D800E0934E03AE81AC3549F4A0910503AA3FBF
:1026E80028F4E0910503EB5FE0930503AE81AD3577
:1026F80031F4AFA5A93018F4EFA5EF5FEFA7AE81CD
:10270800AE3549F4A0914903A93028F4E091490372
:10271800EF5FE0934903AE81AF3559F4AF89B88DC7
:10272800A83BEBE0BE0728F4EF89F88D3196EF8BD4
:10273800F88FAE81A03659F4AD85BE85A83EE3E09A
:10274800BE0728F4ED85FE853A96ED87FE87AE81B3
:10275800A13649F4A0912603AC3328F4E09126036E
:10276800EF5FE0932603AE81A23691F40E948A358A
:10277800A081AA3F21F40E940D36EB5FEC930E94E2
:102788008A35A081AA3F20F40E940D36E65FEC93BB
:102798000E9414360E94163EE02149F0A0911D03C4
:1027A800AA3F28F4E0911D03E65FE0931D030E9411
:1027B80014360E94223EE02149F0A0911E03AA3F50
:1027C80028F4E0911E03E65FE0931E03EAE0EB15B0
:1027D80010F4E894F2F8AB2DEAE00E94F43D0E2ED6
:1027E800A0E0F2FCA1E00E94BD340E94B13509F4DA
:1027F8000EC36894F2F8AE81A13049F4A091170392
:10280800A13028F0E0911703E150E0931703AE815F
:10281800A23049F4A0911803AB3028F0E0911803D6
:10282800E550E0931803AE81A33049F4A091190351
:10283800AD3328F0E0911903E1500E94C235AE8112
:10284800A43049F4A0911B03A53128F0E0911B03A3
:10285800E150E0931B03AE81A53031F4ACA5A13063
:1028680018F0ECA5E150ECA7AE81A63031F4ADA587
:10287800A13018F0EDA5E150EDA7AE81A73031F4F5
:10288800AEA5A13018F0EEA5E150EEA7AE81A830B4
:1028980049F4A0911C03A13028F0E0911C03E150F9
:1028A800E0931C03AE81A93049F4A0914103A13003
:1028B80028F0E0914103E150E0934103AE81AA3052
:1028C80049F4A0914203A13028F0E0914203E1507D
:1028D800E0934203AE81AB3049F4A0914303A130A9
:1028E80028F0E0914303E150E0934303AE81AC301C
:1028F80049F4A0910E03A93128F0E0910E03EC50A1
:10290800E0930E03AE81AD3069F4A0915903B09104
:102918005A03A538E3E0BE0728F00E94ED3231974C
:102928000E947232AE81AE3031F4A8A5A63018F0FC
:10293800E8A5E550E8A7AE81AF3031F4A9A5A630E7
:1029480018F0E9A5E550E9A7AE81A03131F4AAA5B0
:10295800A63018F0EAA5E550EAA7AE81A13131F416
:10296800ACA1A13018F0ECA1E550ECA3AE81A231E6
:1029780031F4ADA1A13018F0EDA1E550EDA3AE8181
:10298800A33131F4AEA1A13018F0EEA1E550EEA3C9
:10299800AE81A43161F4A0916903B0916A030E94E9
:1029A8006C3F28F40E942C327E970E949032AE81B0
:1029B800A53189F4A0910E03EAE0EA9FF001E654FC
:1029C800F040AB89BC89EA17FB0728F4EB89FC893E
:1029D8003197EB8BFC8BAE81A63149F4A091330380
:1029E800A13028F0E0913303E150E0933303AE8146
:1029F800A73149F4A0913503A23028F0E0913503BE
:102A0800E150E0933503AE81A83149F4A091340335
:102A1800A13028F0E0913403E150E0933403AE8113
:102A2800A93149F4AB85BC85129728F0EB85FC8564
:102A38003197EB87FC87AE81AA3159F40E94DC35C7
:102A4800A73DE1E0BE0728F00E94AC3531970E940F
:102A5800E135AE81AB3191F40E946E31AB30E0E0EC
:102A6800BE07E0E08E07E0E09E0740F00E943631A6
:102A7800E150F040604070400E948732AE81AC3136
:102A880059F4A0E023FCA1E0A13030F0A0E023FC41
:102A9800A1E00E941A3623F8AE81AD3161F40E949C
:102AA800E6300E946C3F38F40E94C7303197E093BB
:102AB8006103F0936203AE81AE3161F40E94F0309D
:102AC8000E946C3F38F40E94D3303197E0936D0335
:102AD800F0936E03AE81AF3149F4A0910603A230A2
:102AE80028F0E0910603E150E0930603AE81A0329E
:102AF80049F4A0910803A23028F0E0910803E150BE
:102B0800E0930803AE81A13249F4A0910903A130F2
:102B180028F0E0910903E150E0930903AE81A23265
:102B280049F4A0910A03A13028F0E0910A03E1508A
:102B3800E0930A03AE81A33249F4A0910B03A130BC
:102B480028F0E0910B03E150E0930B03AE81A4322F
:102B580049F4A0910C03A13028F0E0910C03E15056
:102B6800E0930C03AE81A53249F4A0912A03A13069
:102B780028F0E0912A03E150E0932A03AE81A632BF
:102B880049F4A0912B03A13028F0E0912B03E150E8
:102B9800E0932B03AE81A73249F4A0912C03A13016
:102BA80028F0E0912C03E150E0932C03AE81A83289
:102BB80049F4A0912D03A13028F0E0912D03E150B4
:102BC800E0932D03AE81A93249F4A0912E03A130E0
:102BD80028F0E0912E03E150E0932E03AE81AA3253
:102BE80049F4A0912F03A13028F0E0912F03E15080
:102BF800E0932F03AE81AB3249F4A0913003A130AA
:102C080028F0E0913003E150E0933003AE81AC321C
:102C180049F4A0913103A13028F0E0913103E1504B
:102C2800E0933103AE81AD3269F40E9400320E9414
:102C3800703F40F40E94E831E150F040604070403D
:102C48000E94F131AE81AE3251F40E94FA350E94F1
:102C58006C3F28F40E94523131970E945731AE815F
:102C6800AF3259F4A0E036FCA1E0A13030F0A0E08A
:102C780036FCA1E00E941A3636F8AE81A03349F43A
:102C8800A0911003A13028F0E0911003E150E093E7
:102C98001003AE81A13331F4AF8DA13018F0EF8D60
:102CA800E150EF8FAE81A23359F4AF85B889A93CC2
:102CB800E0E0BE0728F0EF85F8893197EF87F88BB9
:102CC800AE81A33349F4A0911503A23028F0E09116
:102CD8001503E150E0931503AE81A43341F40E943B
:102CE800FF35A53120F00E940636E150EC93AE8105
:102CF800A53349F4A0914E03A13028F0E0914E038A
:102D0800E150E0934E03AE81AC3549F4A091050340
:102D1800A13028F0E0910503E550E0930503AE816A
:102D2800AD3531F4AFA5A13018F0EFA5E150EFA70C
:102D3800AE81AE3549F4A0914903A13028F0E09165
:102D48004903E150E0934903AE81AF3559F4AF89A7
:102D5800B88DA13DE7E0BE0728F0EF89F88D3197DF
:102D6800EF8BF88FAE81A03659F4AD85BE85A536B8
:102D7800E0E0BE0728F0ED85FE853A97ED87FE87EF
:102D8800AE81A13649F4A0912603A13028F0E09144
:102D98002603E150E0932603AE81A236D1F40E94C7
:102DA8008A35BF01A0810E940D32FB01A081EFEF9F
:102DB8000E94F43DE02121F00E940D36EA50EC9388
:102DC8000E948A35A081AF3F21F40E940D36E5505C
:102DD800EC930E9414360E94163EE02149F0A0911F
:102DE8001D03A13028F0E0911D03EA50E0931D0374
:102DF8000E9414360E94223EE02149F0A0911E0351
:102E0800A13028F0E0911E03EA50E0931E0323FC52
:102E18006FC00E942136AF8D0E947533AF8DE3E0FD
:102E28000E94D63DE02941F00E9421360E94E034FC
:102E38000E947E320E9428360E94E034E0E0F0E0F2
:102E48006EEF72E40E946A3D09F008F40AC00E941D
:102E58003136A0E0B0E080E893E40E94803C0E9414
:102E68002836E0914803F0E0E0939F03F093A00335
:102E78000E943A36A038E0E0BE0754F0E0919F0384
:102E8800F091A003E050F140E0939F03F093A0037A
:102E9800AF8DA33009F10E94E0340E94703F3CF4EA
:102EA8000E943F360E94873C0E94453614C0A0917C
:102EB800F603AA233AF40E943F360E94803C0E94FF
:102EC800453609C0E0E0E093E303E093E403E093D0
:102ED800E503E093E60304C00E9431360E944536BC
:102EE8000E944E36ADE8B3E00E9486310E9450360B
:102EF80023FE45C0EF81F8850E94FD340E941A3FE9
:102F08000E94153FE0E0F0E060E874E40E94253D8F
:102F1800A0E0B0E48CE995E40E94D73CDF01CB0146
:102F2800EF89F88D0E94E9340E942831DF01CB0136
:102F3800E3E3F3E365E872E40E94253D0E94283646
:102F4800A0910F03A13048F4E0E0E093F303E0938D
:102F5800F403E093F503E093F6030E9431360E94F0
:102F68004536E0910603A0910703AE1740F00E9492
:102F78004E36ADE8B3E00E9486310E945036A0E09C
:102F8800F0FCA1E0E0E00E94D63D0E2EE0910603A1
:102F9800A09107030E94EF3DE02109F446C0E091AB
:102FA8002D03E030F1F4A985BA85E0E0F4E00E9451
:102FB8005436A3E9B3E00E948631E0919B03F09177
:102FC8009C030E946636A5E9B3E00E948631E09131
:102FD8009D03F0919E030E946636A7E9B3E00E9424
:102FE8008631A0912D03A130E9F4AF81B885E2E0E4
:102FF800F0E00E94933E3597E0939303F093940397
:10300800E0919B03F0919C033597E0939503F0932F
:103018009603E0919D03F0919E033597E093970303
:10302800F0939803E0E0E0930703F0916F03E0E08A
:10303800DF01E0913903F0E0EA0FFB1FA3ECB3E0F6
:103048000E94CC300E946D36A0E0B0E080E192E4AE
:103058000E94253D7F936F93FF93EF930E94DC3589
:103068000E947636AF91BF918F919F910E94E9346B
:103078000E94D73CE093C303F093C4036093C50355
:103088007093C6030E947B36E0E0F0E060E87FE3DF
:103098000E94903D0E2E0E947B36E0E0F0E068EC46
:1030A80072E40E948A3DE02109F10E946D36A0E099
:1030B800B0E080E09FE30E94873CABEAB3E00E9467
:1030C800163C0E94103F0E946D36E093C703F093B0
:1030D800C8036093C9037093CA030E947B360E9499
:1030E8000932ABE5B3E00E94FE3015C0E0E0E093A2
:1030F800AB03E093AC03E093AD03E093AE03E0933E
:10310800C703E093C803E093C903E093CA03E093BD
:103118005B03E0935C030E9492310E941E310E947F
:10312800903DEF930E9484360E94903DAF91EA2330
:10313800C1F10E941531E0E0F0E068EC72E40E9411
:10314800253D0E946E310E941F3F0E9428310E9437
:103158008636A091BF03B091C0038091C1039091BE
:10316800C203E0E0F0E064E172E40E94D73CDF01D2
:10317800CB010E94A9310E94253DA0E0B0E080E289
:1031880091E40E94D73C0E948636E091BF03F091FB
:10319800C0036091C1037091C203DE0114960E94BE
:1031A80086310E946633A0912403EDEF0E94F43D1E
:1031B8000E220E941A34E02129F0E0912403EF5FE7
:1031C800E0932403A62D0E947C35A0912403EFEF01
:1031D8000E94F43D0E220E941A34E02129F0E8945E
:1031E800F0F8E0E0E0932403A0912403EEE10E94CC
:1031F800D63D0E2E0E941A34E02119F0E1E0E0934A
:103208002703E0912603E03019F4E0E0E093270378
:103218000E948F360E944935A0912703E0E00E9462
:10322800F93DE02119F0E1E0E0932703A09127039D
:10323800AC3321F4EFEFF0E0E98FFA8FA0910503AA
:10324800A13028F0E0910503F0E00E944133A091FD
:1032580031030E9475330E943835E02159F1EE8D13
:10326800EF5FEE8FF0E03196BF01A98DBA8D0E9415
:103278007636E617F70790F40E9494360E94303E9F
:103288000E2E0E94A136E4EAF1E060E070E00E94B0
:10329800283EE02919F0E0E0E98FEA8FA98DBA8D80
:1032A8000E947636AE8DB0E0EA17FB0710F4E0E036
:1032B800EE8F02C0E0E0EE8F0E9438350E2E0E949D
:1032C80094360E94403E0E22AF85B889E4EAF1E0C8
:1032D8000E94043EE02151F0A98DBA8DA639E0E0A4
:1032E800BE0720F4E6E9F0E0E98FFA8FEF8DE030D1
:1032F80009F086C0442041F5E0911403E03041F420
:10330800E12FF0E034960E941333EA0FFB1F03C04D
:103318000E9482333F96A98DBA8D0E94AA36AEE3E9
:103328000E94A830A4E00E94A830E0911403E03085
:1033380011F4A12F01C0ABE00E94A830A0E00E94C8
:10334800B136A98D0E94B736E1E0E41509F058C0FE
:103358004424A0911903B0E0E2E0F0E00E94933E1B
:10336800E0931A03F0E0BC96DF01E0911603F0E069
:10337800AE0FBF1FE0911703F0E0AE0FBF1FE09143
:1033880018030E94C236AE0FBF1FECA5F0E0AE0FC7
:10339800BF1FEDA5F0E0AE0FBF1FEEA5F0E0AE0F2A
:1033A800BF1FE0911C030E94C936F0E0AE0FBF1F9B
:1033B800E0914303F0E00E94AA36AEE30E94A830F1
:1033C800ACE20E94D436A09118030E94A830A091C4
:1033D8001A030E94DE36ACA50E94A830ADA50E9453
:1033E800A830AEA50E94E436A09141030E94A830FF
:1033F800A09142030E94A830A09143030E94B736CF
:10340800AF8DA13009F06DC0A98DBA8DA93CE0E05F
:10341800BE0720F0E8ECF0E0E98FFA8FE0911B039B
:10342800AFE2AE27E1E0AE27E6E3EA277E2FA98DDB
:10343800BA8DE5E00E94703EE7277E2F8F2F0E940D
:103448001333E5E00E94703EA72FB82FAE27BF27A1
:10345800E1E0F0E0AE27BF27E6E3F0E0AE27BF27C4
:10346800E0911803F0E0AE27BF27E12FF0E0AE2788
:10347800BF27E1E0F0E0EA27FB27E0935D03F09344
:103488005E03AFE20E94A830A1E00E94A830A0E04D
:103498000E94DE360E94EA36A98DBA8DE5E00E94C8
:1034A800703EE98FFA8FAA8D0E94A830A98D0E94DC
:1034B800A8300E941333E5E00E94703E0E94413319
:1034C800E0915003AE2F0E94B1360E94EA36A0E088
:1034D8000E94A830A09118030E94A830A12F0E9432
:1034E800F036AF8DA33009F092C0442009F045C0F2
:1034F800E0911403E03051F4E12FF0E03596DF015C
:10350800E0914403F0E0AE0FBF1F05C0E091440313
:10351800F0E07096DF01E0914503F0E0AE0FBF1FC9
:10352800E0914603F0E0EA0FFB1F0E941333EA0F15
:10353800FB1FA98DBA8D0E94AA36AEE60E94A8305C
:10354800A5E00E94A830E0911403E03011F4A12F07
:1035580001C0ABE00E94A830A09144030E94A830AB
:10356800A09145030E94A830A09146030E94B1365D
:10357800A98D0E94F6360E94F036E1E0E41509F0C4
:1035880046C04424E0911603F0E0BD96DF01E091C7
:1035980017030E94C9360E94C236AE0FBF1FD296CB
:1035A800E0911C03F0E0AE0FBF1FE0911503F0E0BF
:1035B800EA0FFB1F7E2F8F2FAB85BC85EAE00E94A8
:1035C800703EE70FF81FE0935D03F0935E03AEE6ED
:1035D8000E94A830ADE20E94D436A09142030E9416
:1035E800A830A09141030E94DE36A2E30E94F6367D
:1035F8000E94E436EB85AAE0EA9FF001AE2F0E9414
:10360800A830A09115030E94F6360E94F0360E9459
:10361800FD360E941232FF27662777270E94763FE1
:1036280034F4E091AB03A6E3B0E00E94553F0E945A
:1036380002370E94E034FF27662777270E944D3C17
:103648000E946A3D09F008F408C00E943136A7E3D9
:10365800B0E00E94143C0E94553F0E9407370E9428
:103668003A36F0E0EA17FB0734F4E0919F03A8E349
:10367800B0E00E94553F0E940C370E9411370E940B
:10368800CC3D0E94383E0E2E0E941137E8ECF0E047
:1036980060E070E00E94403EE02141F0E091B30319
:1036A800F091B403A1E5B0E00E944D3F0E941A37A3
:1036B8000E9411370E94CC3D0E94763F44F4E0916D
:1036C800B303F091B403A3E5B0E00E944D3F0E941C
:1036D8001F37A0919303B0919403EA17FB0744F4B2
:1036E800E0919303F0919403A7E5B0E00E944D3F69
:1036F8000E942437A0919503B09196030E94103E32
:103708000E944B340E942334E02141F0E09195035C
:10371800F0919603A9E5B0E00E944D3F0E94293739
:10372800A0919703B09198030E94103E0E944B34D9
:103738000E942334E02141F0E0919703F09198032F
:10374800ABE5B0E00E944D3F0E9495320E942331C4
:10375800AE1BBF0BA436E0E0BE0710F00E94733525
:10376800E091B303F091B4036091B5037091B6038F
:103778000E94E0340E944D3C0E94D73CA1EAB3E08D
:103788000E9486310E942E370E943337E093A103AE
:10379800F093A2030E9438370E942E37EA17FB07DE
:1037A80044F4E091A103F091A203A5E5B0E00E94E2
:1037B8004D3F033608F0DAC70E94A6350081A09174
:1037C8003703A13048F420FC07C0A0E0F799A1E036
:1037D800EA2FE295E07F19C0A0E0F799A1E0EA2F6F
:1037E800E295E07F0E2EA0E0F399A1E0EA2FEE0F1C
:1037F800EE0F0E0EA0E0F499A1E0EA2FEE0FA02D37
:10380800AE0FE0E0F599E1E0EA0FE8AB0E94E034A2
:10381800EDECFCEC6CEC7DEB0E946A3D18F4E8A939
:10382800E05AE8ABEAE00E943D37EAE0DE01AC5B33
:10383800BF4FEC930E9442370E944837EAE00E944B
:103848004D37EAE00E945237EAE00E9457370E945B
:103858005C37E89435F8A0E031FCA1E00E947533AC
:10386800A0E032FCA1E0E1E00E94D63D0E2AA0E0F3
:1038780034FCA1E0E1E00E94D63DE02911F020FAF5
:1038880001C0E894F5F8E0912F03E03021F40E949C
:103898007E370E948E37A0912F03A13081F4A0E0DB
:1038A80022FCA1E0EA2FEE0FE75F0E2EA0E022FC3B
:1038B800A1E0EA2FEE0FEE0FE00D0E949D37A091D8
:1038C8002F03A23099F40E947E37A0E022FCA1E0E9
:1038D800EA2F0E94AD370E0EA0E022FCA1E0EA2FED
:1038E800E295E07FEE0F0E0E0E948E37A0912F0317
:1038F800A33031F4E0E022FCE1E0E85F0E949D376C
:10390800A0910E03A83109F041C00E94B237A23D30
:10391800E0E0BE07E0E08E07E0E09E071CF0E1E093
:10392800E09301030E941137A83FE0E0BE07E0E002
:103938008E07E0E09E071CF0E3E0E09301030E949D
:103948001137AF3FE0E0BE07E0E08E07E0E09E07FA
:103958001CF0E7E0E09301030E941137A430E1E096
:10396800BE07E0E08E07E0E09E071CF0EFE0E09382
:1039780001030E941137AE30E1E0BE07E0E08E0798
:10398800E0E09E071CF0EFE1E0930103A0910E0335
:10399800A43209F041C00E94B237A633E1E0BE0765
:1039A800E0E08E07E0E09E071CF0E1E0E093010311
:1039B8000E941137AA34E1E0BE07E0E08E07E0E09C
:1039C8009E071CF0E3E0E09301030E941137AE3537
:1039D800E1E0BE07E0E08E07E0E09E071CF0E7E0CC
:1039E800E09301030E941137A836E1E0BE07E0E04A
:1039F8008E07E0E09E071CF0EFE0E09301030E94D1
:103A08001137AC37E1E0BE07E0E08E07E0E09E0743
:103A18001CF0EFE1E0930103A0910E03A03309F03D
:103A280041C00E94B237A638E1E0BE07E0E08E0749
:103A3800E0E09E071CF0E1E0E09301030E941137EB
:103A4800AC3CE1E0BE07E0E08E07E0E09E071CF03A
:103A5800E3E0E09301030E941137A63DE1E0BE07D1
:103A6800E0E08E07E0E09E071CF0E7E0E09301034A
:103A78000E941137A03EE1E0BE07E0E08E07E0E0DB
:103A88009E071CF0EFE0E09301030E941137AF3E60
:103A9800E1E0BE07E0E08E07E0E09E071CF0EFE102
:103AA800E0930103A0911403A13081F4A0E020FC6D
:103AB800A1E0EA2F0E94AD370E2EA0E020FCA1E085
:103AC800EA2FE295E07FEE0FE00D4E0FA091020382
:103AD800A431F0F40E9412320E94B8376CF0FE0153
:103AE800EE5BFF4F3396FF93EF930E94C0370E941F
:103AF800C637AF91BF91EC930E94D137FF93EF93F4
:103B08000E94C0370E94D73EAF91BF91EC930DC081
:103B180020FE05C0E0E40E94D637E0E402C00E941F
:103B28004237DE01AA5BBF4FEC93AD8DA13090F018
:103B3800ED8DE150ED8FE8E70E94D637E091140350
:103B4800E03029F4FE01EE5BFF4F148303C0E0E58B
:103B58000E944837AC8DA13058F0EC8DE150EC8FC5
:103B6800E8E30E94D6370E94D137A0913203A083A0
:103B7800AB8DA13048F0EB8DE150EB8FE9E30E946B
:103B8800D637E0E50E944837E0911103E03019F597
:103B98004058A0918E03AA2392F4E0E40E943D3796
:103BA800A0918D03B0918E03AD39EFEFBE0714F4E9
:103BB800689435F80E94DB370E94E33702C0E89426
:103BC80035F80E94E8371A9724F00E94ED370E94D2
:103BD800F4370E94FC37A0911103A13009F045C0C9
:103BE800E8A9E85FE8AB0E940938FF2392F4E0E413
:103BF8000E943D370E940938E73FAFEFFA0714F4F7
:103C0800689401C0E89435F80E9409380E94A03DE4
:103C180004C0E89435F80E940938E0938F03F093C4
:103C280090030E94E8371A9724F00E94ED370E940B
:103C3800F4370E94FC370E940938BF01DF01E3E630
:103C4800F0E00E94103E0E2EDB01EDE9FFEF0E942E
:103C58000A3EE02951F0E89435F8E0E40E943D3747
:103C6800E0E4DE01AC5BBF4FEC930E941538FF9394
:103C7800EF930E9411370E941A380E94C637AF91FD
:103C8800BF910E941F383696FF93EF930E94243805
:103C98000E94C637AF91BF910E941F383796FF9395
:103CA800EF930E9424380E94D73EAF91BF91EC93C6
:103CB8000E941137A639E0E0BE07E0E08E07E0E099
:103CC8009E0764F4E0E40E944D37E0E40E94523716
:103CD800E0E40E945737E0E0E0930103013009F087
:103CE8005BC00E942A380E943238A83EE3E0BE0733
:103CF800B8F0505E0E9437380E943D380E941F3845
:103D08003E96BF010E9432380E9448380E941F38F0
:103D18003F96BF010E9432380E947636DF011BC0F1
:103D280050560E943238A436E0E0BE0728F00E94C0
:103D380037380E944838EC930E945338BF010E94DC
:103D480032380E9476360E9458380E941F383F96B3
:103D5800BF010E943238EAE0F0E00E945F38A0918B
:103D68000003AA3010F00E9464380E946A38A091BB
:103D780000030E9470380E941F383A96BF01AC2D8C
:103D8800B0E00E9433370E94F4370E947738BF01B1
:103D9800AC2D0E947038EC93023009F06DC0505C75
:103DA8000E940032A03AE6E8BE07E1E08E07E0E0B4
:103DB8009E0778F00E947C38FF93EF930E940032B0
:103DC800E0EAF6E861E070E00E948138AF91BF91C7
:103DD800EC930E9400320E948C3878F00E94773869
:103DE800FF93EF930E940032E0E1F7E260E070E0B9
:103DF8000E948138AF91BF91EC930E9400320E94DB
:103E0800943868F00E949C38FF93EF930E94003228
:103E18000E9415340E948138AF91BF91EC930E94A3
:103E280000320E94A13868F00E94A938FF93EF93EE
:103E38000E9400320E941A380E948138AF91BF91C7
:103E4800EC930E9400320E94B83758F00E94533811
:103E5800FF93EF930E94AE380E948138AF91BF91D3
:103E6800EC930E94B438FF93EF930E94AE380E94FF
:103E7800D33EAF91BF91EC93033009F08FC0E7E7D1
:103E88000E94B938A091BA03AA2392F4E091B7032B
:103E9800F091B8036091B9037091BA030E94A43DF0
:103EA800E093B703F093B8036093B9037093BA0330
:103EB8000E9484360E942831772312F40E94C33866
:103EC8000E9484360E9428310E94C93810F40E944A
:103ED800D2380E9484360E9428310E94D83810F4C3
:103EE8000E94E1380E9484360E9428310E94E738F7
:103EF80010F40E94EA380E94F0380E948C387CF056
:103F08000E947738FF93EF930E94F038E0E1F7E2E0
:103F180060E070E00E94C637AF91BF91EC930E94B9
:103F2800F0380E9494386CF00E949C38FF93EF930D
:103F38000E94F0380E9415340E94C637AF91BF9195
:103F4800EC930E94F0380E94A1386CF00E94A938C6
:103F5800FF93EF930E94F0380E941A380E94C637E8
:103F6800AF91BF91EC930E94F0380E94B8375CF093
:103F78000E945338FF93EF930E94F9380E94C63786
:103F8800AF91BF91EC930E94B438FF93EF930E94D6
:103F9800F9380E94D73EAF91BF91EC93043009F0F5
:103FA80054C05058EEE30E94B938A0918A03AA235E
:103FB80012F40E94FF380E940A39772312F40E94F3
:103FC800C3380E940A390E94C93810F40E94D238B6
:103FD8000E940A390E94D83810F40E94E1380E94E1
:103FE8000A390E94E73810F40E94EA380E94103912
:103FF800A031E7E2BE0724F00E9477380E94153905
:104008000E941039A83EE3E0BE0724F00E949C38C5
:104018000E941C390E941039A436E0E0BE0724F043
:104028000E94A9380E9423390E9410391A974CF02F
:104038000E945338BF010E9410390E9433370E94F2
:10404800F4370E94B4380E942A39053071F5505867
:10405800EEE30E94B9380E943339A091EA03AA23FB
:1040680012F40E94D2380E949231E0E0F0E066EC4F
:1040780072EC0E946A3D10F40E94E1380E943939BE
:10408800A436E0E0BE0724F00E94A9380E943E3919
:104098000E945338BF010E9439390E9433370E9469
:1040A800F4370E94B4380E9445390630A1F55058BB
:1040B800E0E00E944E39E5E00E945339E8E70E94AB
:1040C8005839AC81BD81A83EE3E0BE073CF00E94B0
:1040D8009C38BF01AC81BD810E945D39AC81BD8136
:1040E800A436E0E0BE073CF00E94A938BF01AC81CD
:1040F800BD810E9462390E945338BF01AC81BD81E5
:104108000E9433370E94F4370E94B438BF01AC8153
:10411800BD810E946739073009F076C0A98DBA8D34
:104128000E946C3F30F5ECE00E944E390E946E39D7
:10413800E436A0E0FA0740F00E947C38BF01A98D60
:10414800BA8D0E947339EC930E946E393A9740F009
:104158000E947738BF01A98DBA8D0E947839EC93F7
:104168000E949C38BF010E946E390E945838EC9317
:104178004BC0E0914203E03029F5EBE00E944E3954
:104188000E947D39E436A0E0FA0740F00E947C38AE
:10419800BF01A989BA890E947339EC930E947D39BD
:1041A8003A9740F00E947738BF01A989BA890E94DE
:1041B8007839EC930E949C38BF010E947D390E9497
:1041C8005838EC93A0914203A130F1F4EBE00E943F
:1041D8004E39A989BA89A436E0E0BE0740F00E94AA
:1041E8007C38BF01A989BA890E944838EC930E949B
:1041F8007738BF01A989BA890E9476360E94583853
:10420800EC93E7E70E948239083009F07EC00E94EB
:104218002A38A0918503B0918603A135EBEFBE073C
:1042280034F4E1E5FBEFE0938503F0938603A09176
:104238008503B0918603A03BE4E0BE0734F0EFEAC3
:10424800F4E0E0938503F0938603A0918603AA2304
:104258004AF40E94E138E0918503F09186030E94B8
:10426800A03D04C0E0918503F0918603E0938703A5
:10427800F0938803A0918703B0918803ECE3F0E002
:104288000E94933EE0936303F09364030E9487398E
:10429800ECE30E94703EA0918703B0918803AE1BA7
:1042A800BF0BA0936503B093660324FE25C00E944C
:1042B80087391A9710F00E9464380E946A380E9461
:1042C8008739EAE0F0E00E94C23EDB010E941F3815
:1042D8003A96BF01A0916503B09166030E947636B5
:1042E8000E9458380E941F383B96BF01A091650371
:1042F800B09166030E948C39E3E70E948F39E8E3A6
:104308000E949439E4E50E949939093009F056C0B1
:1043180050580E946438EEE30E94B938A0918A038D
:10432800AA2312F40E94FF380E940A39772312F454
:104338000E94C3380E940A390E94C93810F40E94AA
:10434800D2380E940A390E94D83810F40E94E13805
:104358000E940A390E94E73810F40E94EA380E9445
:104368001039A031E7E2BE0724F00E9477380E9496
:1043780015390E941039A83EE3E0BE0724F00E94D8
:104388009C380E941C390E941039A436E0E0BE0710
:1043980024F00E94A9380E9423390E9410391A97E4
:1043A8004CF00E945338BF010E9410390E943337E5
:1043B8000E94F4370E94B4380E942A390A30F9F46E
:1043C80050580E946438EEE30E94B9380E9433398D
:1043D8000E943939A436E0E0BE0724F00E94A938CB
:1043E8000E943E390E945338BF010E9439390E9409
:1043F80033370E94F4370E94B4380E9445390B3095
:10440800A1F55054E9E30E945339E8E30E94583972
:104418000E94FA35A83EE3E0BE0740F00E949C38AF
:10442800BF010E94FA350E943D38EC930E94FA358C
:10443800A436E0E0BE0740F00E94A938BF010E9400
:10444800FA350E944838EC930E945338BF010E9405
:10445800FA350E9476360E9458380E941F383F96D7
:10446800BF010E94FA350E948C390C3009F073C0E4
:104478000E946438EEE30E944E390E942E37E0E035
:10448800F0E00E949E39E6EFFFEF0E94103EE02127
:1044980011F00E94C3380E942E37E7EFFFEF0E9409
:1044A8009E39ECE9FFEF0E94103EE02111F00E94D6
:1044B800D2380E942E37EDE9FFEF0E949E39E8E1DD
:1044C800FCEF0E94103EE02111F00E94E1380E94AA
:1044D8002E37A931ECEFBE0714F40E94EA38A091F8
:1044E800A203AA2352F4E091A103F091A2030E942F
:1044F800A03DE093A103F093A2030E942E37A83EAB
:10450800E3E0BE073CF00E949C38BF010E942E37B2
:104518000E945D390E942E37A436E0E0BE073CF0C9
:104528000E94A938BF010E942E370E9462390E945A
:104538002E371A974CF00E945338BF010E942E372D
:104548000E9433370E94F4370E94B438BF010E949A
:104558002E370E946739AAA10E940D32A9A1E0E076
:104568000E94F93DE02909F4AFC05F77E091380374
:10457800E170EE0F4E23E0913803E6950E94A239D0
:104588000E2EE0913803E695E695E170AE2FE0E057
:10459800F5FCE1E0EA2BEE0FEE0FE00D4E0F0E9466
:1045A8005C37A9A10E940D32AAA1E0E00E94F93D62
:1045B800E02159F1A9A1A13029F40E94A739ECE022
:1045C8000E948239A9A1A23029F40E94A739EDE0FE
:1045D8000E948239A9A1A33029F40E94A739EBE0EF
:1045E8000E9482390E94AA3929F00E94A739ECE07A
:1045F8000E9482390E9451330E94B43929F00E94E6
:10460800A739EBE00E9482392AC0A9A1A13029F478
:104618000E94BA39ECE00E949939A9A1A23029F484
:104628000E94BA39EDE00E949939A9A1A33029F472
:104638000E94BA39EBE00E9499390E94AA3929F000
:104648000E94BA39ECE00E9499390E9451330E94C5
:10465800B43929F00E94BA39EBE00E949939AAA12D
:10466800A13029F40E94BE39ECE00E949939AAA130
:10467800A23029F40E94BE39EDE00E949939AAA11E
:10468800A33029F40E94BE39EBE00E949939AAA10F
:10469800E4E00E94D63D0E94B43929F00E94BE3958
:1046A800ECE00E949939AAA1E5E00E94D63D0E945B
:1046B800B43929F00E94BE39EBE00E949939E091A3
:1046C8001103E03009F44058E0914A03A0919303A4
:1046D800B09194030E94C2390E2EA0914A030E9401
:1046E800C63931F0E0E00E94CB39E0E00E94CF39D2
:1046F800A0919503B0919603E0914B030E94C239B3
:104708000E2EA0914B030E94C63931F0E1E00E94C1
:10471800CB39E1E00E94CF39A0919703B09198037B
:10472800E0914C030E94C2390E2EA0914C030E94C6
:10473800C639C1F0E2E00E94CB39E2E00E94533969
:10474800E0E00E945839E9E70E948239E0E50E94DA
:104758008F39E0E50E949439E0E00E949939E1E060
:10476800E0933F03F29B02C04B7F4F5F033611F08B
:104778000C949F2C31E0303140F40E94DE39EAE09D
:10478800EC93E89435F83F5FF6CFAE81EBE50E94F5
:10479800E639EAE50E94D63DE02911F0E5E3EE832B
:1047A800AE81A63311F4ECE5EE83EE81E03029F416
:1047B800E0911603F0E0ED8BFE8BAE81A13029F479
:1047C800E0911703F0E0ED8BFE8BAE81A23029F467
:1047D800E0911803F0E0ED8BFE8BAE81A33029F455
:1047E800E0911903F0E0ED8BFE8BAE81A43029F443
:1047F800E0911B03F0E0ED8BFE8BAE81A53021F438
:10480800ECA5F0E0ED8BFE8BAE81A63021F4EDA592
:10481800F0E0ED8BFE8BAE81A73021F4EEA5F0E041
:10482800ED8BFE8BAE81A83029F4E0911C03F0E0FB
:10483800ED8BFE8BAE81A93029F4E0914103F0E0C5
:10484800ED8BFE8BAE81AA3029F4E0914203F0E0B3
:10485800ED8BFE8BAE81AB3029F4E0914303F0E0A1
:10486800ED8BFE8BAE81AC3029F4E0910E03F0E0C5
:10487800ED8BFE8BAE81AD3021F40E94ED32ED8BD5
:10488800FE8BAE81AE3021F4E8A5F0E0ED8BFE8B17
:10489800AE81AF3021F4E9A5F0E0ED8BFE8BAE815F
:1048A800A03121F4EAA5F0E0ED8BFE8BAE81A131B9
:1048B80021F4ECA1F0E0ED8BFE8BAE81A23121F466
:1048C800EDA1F0E0ED8BFE8BAE81A33121F4EEA1DA
:1048D800F0E0ED8BFE8BAE81A43121F40E942C32E6
:1048E800ED8BFE8BAE81A53121F4EB89FC89ED8B34
:1048F800FE8BAE81A63129F4E0913303F0E0ED8B15
:10490800FE8BAE81A73129F4E0913503F0E0ED8B01
:10491800FE8BAE81A83129F4E0913403F0E0ED8BF1
:10492800FE8BAE81A93121F4EB85FC85ED8BFE8BE6
:10493800AE81AA3121F40E94AC35ED8BFE8BAE819D
:10494800AB3131F4E0917B03F0917C03ED8BFE8B6E
:10495800AE81AC3131F4E0E023FCE1E0F0E0ED8B36
:10496800FE8BAE81AD3121F40E94C730ED8BFE8BFA
:10497800AE81AE3121F40E94D330ED8BFE8BAE8137
:10498800AF3129F4E0910603F0E0ED8BFE8BAE81A8
:10499800A03229F4E0910803F0E0ED8BFE8BAE81A4
:1049A800A13229F4E0910903F0E0ED8BFE8BAE8192
:1049B800A23229F4E0910A03F0E0ED8BFE8BAE8180
:1049C800A33229F4E0910B03F0E0ED8BFE8BAE816E
:1049D800A43229F4E0910C03F0E0ED8BFE8BAE815C
:1049E800A53229F4E0912A03F0E0ED8BFE8BAE812D
:1049F800A63229F4E0912B03F0E0ED8BFE8BAE811B
:104A0800A73229F4E0912C03F0E0ED8BFE8BAE8108
:104A1800A83229F4E0912D03F0E0ED8BFE8BAE81F6
:104A2800A93229F4E0912E03F0E0ED8BFE8BAE81E4
:104A3800AA3229F4E0912F03F0E0ED8BFE8BAE81D2
:104A4800AB3229F4E0913003F0E0ED8BFE8BAE81C0
:104A5800AC3229F4E0913103F0E0ED8BFE8BAE81AE
:104A6800AD3231F4E0917703F0917803ED8BFE8B52
:104A7800AE81AE3221F40E945231ED8BFE8BAE81B5
:104A8800AF3231F4E0E036FCE1E0F0E0ED8BFE8B94
:104A9800AE81A03329F4E0911003F0E0ED8BFE8B9A
:104AA800AE81A13321F4EF8DF0E0ED8BFE8BAE816A
:104AB800A23321F4EF85F889ED8BFE8BAE81A33309
:104AC80029F4E0911503F0E0ED8BFE8BAE81A43361
:104AD80049F4E0912C03F0E0E65BFC4FE081F0E064
:104AE800ED8BFE8BAE81A53329F4E0914E03F0E007
:104AF800ED8BFE8BAE81AC3529F4E0910503F0E037
:104B0800ED8BFE8BAE81AD3521F4EFA5F0E0ED8B9A
:104B1800FE8BAE81AE3529F4E0914903F0E0ED8BD0
:104B2800FE8BAE81AF3521F4EF89F88DED8BFE8BCE
:104B3800AE81A03621F4ED85FE85ED8BFE8BAE812E
:104B4800A13629F4E0912603F0E0ED8BFE8BAE81CF
:104B5800A23631F40E948A35E081F0E0ED8BFE8BBD
:104B68000E9414360E94163EE02129F0E0911D03B0
:104B7800F0E0ED8BFE8B0E9414360E94223EE0216D
:104B880029F0E0911E03F0E0ED8BFE8BAE81E0E0B2
:104B98000E94E639E3E00E94EB39E1E10E94EB393B
:104BA800E2E10E94EB39E3E10E94EB39E5E10E9482
:104BB800EB39EAE10E94EB39EBE10E94EB39EDE1D8
:104BC8000E94EB39EEE20E94D63DE0291E2E0E949B
:104BD800F0390E94043EE0211E2AAE81EEE50E94D3
:104BE800D63D0E2EA0914903E2E00E94F93D0E2227
:104BF800E5E00E94F43DE021E12911F0F69A01C0B8
:104C0800F698A0E0F699A1E0EA2FE795E0E0E795AD
:104C18005E2F40E0E0E0E8ABE0930103FE01EE5BCD
:104C2800FF4F3396BF01AE81B0E0A7FDBFEF0E94F2
:104C380033370E94F4370E94D137BF01AE81B0E00C
:104C4800A7FDBFEF0E946739AD89BE89A031E7E2B1
:104C5800BE0740F00E947738BF01AD89BE890E9427
:104C6800FA39EC93AD89BE89A83EE3E0BE0740F06F
:104C78000E949C38BF01AD89BE890E943D38EC93E3
:104C8800AD89BE89A436E0E0BE0740F00E94A9388D
:104C9800BF01AD89BE890E944838EC93AD89BE89B1
:104CA8001A9738F00E9453380E94FF390E945838EA
:104CB800EC930E94B438BF01AD89BE890E948C393B
:104CC800EE81E03079F4ECE10E94033AE0E50E94DD
:104CD8005737EDE60E945339E4E50E945839E0E57C
:104CE8000E948239AE81A13031F4EBE50E94033A8B
:104CF800EDE60E945737AE81A23029F40E94063AA9
:104D0800E8E30E945737AE81A33049F4EEE50E94EC
:104D18004D37E0E30E945237E7E70E945737AE81EC
:104D2800A83011F40E940A3AAE81AC3031F4EEE3B7
:104D38000E94103AECE70E945737AE81E1E10E94E9
:104D4800E639E2E10E94EB39E3E10E94EB39E5E163
:104D58000E94EB39EDE10E94EB39EEE20E94D63D6C
:104D6800E02939F00E9453380E94FF390E945838D0
:104D7800EC93E7EAE0937A000E940933E7E2E093D4
:104D88007A000E94133AEEE00E94EB39E1E10E94BA
:104D9800D63DE02911F0E1E07E2EAE81E6E00E94EA
:104DA800E639EFE00E94EB39E2E10E94D63DE029C6
:104DB80011F0E2E07E2EAE81E7E00E94E639E0E104
:104DC8000E94EB390E94163A11F0E3E07E2E0E9411
:104DD8001333D39708F45DC00E9482330E9487334F
:104DE800E72D0E948E3320F0E8ECF0E00E9441337A
:104DF800A0914203A13011F40E949E33E72D0E9436
:104E0800A9330E941B3AAC91A13008F441C00E941A
:104E1800223A0E94C9330E947B3F4CF40E941B3AFD
:104E28000E942B3A0E94963D0E94353A23C00E9468
:104E38003E3A0E94EA33EF930E943E3A0E94F333CF
:104E4800AF91EA2379F00E941B3A0E942B3A0E9404
:104E58009B3DA093A703B093A8038093A9039093C5
:104E6800AA0308C00E943E3A0E94FC331CF00E942C
:104E7800403A0EC0A091A703B091A8038091A9035E
:104E88009091AA030E9415340E94BD3E0E944133AE
:104E980004C00E9446330E94403AAE81AD3029F5E5
:104EA8000E941538FF93EF930E94A1360E941A388A
:104EB8000E94C637AF91BF910E941F383696FF9364
:104EC800EF930E944F3A0E94C637AF91BF910E945C
:104ED8001F383796FF93EF930E944F3A0E94D73EB0
:104EE800AF91BF91EC93E0E2E8ABAE81A53141F41C
:104EF800EEE30E944D37ECE00E945237E0E6E8AB63
:104F08000E94133AEEE00E94EB39E1E10E94D63D9F
:104F1800E029B1F00E94553AE4E00E94593A28F09D
:104F28000E9415380E945F3AEC930E9413331A9737
:104F380028F00E94623A0E945838EC930E94693A1D
:104F4800AE81E6E00E94E639EFE00E94EB39E2E14B
:104F58000E94D63DE029B1F00E94553AE2E00E9455
:104F6800593A28F00E9415380E945F3AEC930E9443
:104F780013331A9728F00E94623A0E945838EC932B
:104F88000E94693AAE81E7E00E94E639E0E10E94BA
:104F9800EB390E94163AB1F00E94553AE1E00E94BE
:104FA800593A28F00E9415380E945F3AEC930E9403
:104FB80013331A9728F00E94623A0E945838EC93EB
:104FC8000E94693AAE81E5E00E94703A1E2EAE81D9
:104FD800E6E00E94703A1E2AAE81E7E00E94703A2D
:104FE800E12951F1E72DF0E0DE019B96AE0FBF1FDE
:104FF800EC91F0E0AB85BC850E94483EDF01E4E619
:10500800F0E00E94803E0E9441330E9413331A97B9
:1050180050F00E941538BF010E9413330E94763663
:105028000E945838EC930E94763A0E9413330E94EB
:105038008C39E7E70E945737AE81A431B1F40E945A
:1050480015380E947C3A0E9448380E941F383696CC
:105058000E947C3A0E9476360E9458380E941F3877
:1050680037960E947C3A0E948C39AE81A63129F489
:105078000E940A3AEBE00E944E39AE81A73129F42A
:105088000E940A3AE0E40E944E39AE81A83129F420
:105098000E940A3AECE00E944E39AE81A931D1F45F
:1050A800A091F603AA2322F40E94DB370E94E3377B
:1050B8000E941538BF010E94E8370E9433370E94CA
:1050C800F4370E94763A0E94E8370E946739E7E78A
:1050D8000E945737AE81AA31F1F40E94823AA43671
:1050E800E0E0BE0740F00E941538BF010E94823AF6
:1050F8000E944838EC930E94763A0E94823A0E94B5
:1051080076360E9458380E941F383796BF010E9491
:10511800823A0E948C39AE81AB3169F4ECE70E9487
:10512800103AE8E70E9457370E9453380E94FF3927
:105138000E945838EC93AE81AC3149F4E0E30E9408
:105148004D37EDE60E945237E4E50E945737AE81AD
:10515800AF3149F4EEE30E944D37EDE60E94523735
:10516800E3E70E945737AE81A53229F40E94873AB7
:10517800E5E00E945737AE81A63229F40E94873AAB
:10518800E8E00E945737AE81A73229F40E948B3A93
:10519800E3E60E945737AE81A83229F40E948B3A81
:1051A800E8E70E945737AE81A93249F4E7E70E9441
:1051B8004D37E0E40E945237E8E70E945737AE8146
:1051C800AB3231F4E9E30E948F3AEEE00E945737A0
:1051D800AE81AC3231F4ECE70E948F3AEDE60E94E2
:1051E8005737AE81AD3231F4E0E00E94923AE0E008
:1051F8000E945737AE81EDE10E94E639EEE10E9448
:10520800D63DE02921F1E3E70E944E39E8E30E9408
:105218005339AE81AD3111F4EEE501C0E8E7DE01A6
:10522800A35BBF4FEC930E94953A1A9748F00E94EF
:10523800763A0E94953A0E9476360E945838EC9346
:105248000E949A3ABF010E94953A0E948C390E94A6
:10525800133AE6E00E94EB39E7E00E94D63DE029E8
:1052680019F0E3E70E944E39AE81EEE00E94E6397C
:10527800EFE00E94EB39E0E10E94D63DE02949F0D9
:10528800EDE60E944E39E9E70E945339E4E50E94B1
:105298005839AE81E1E10E94E639E2E10E94EB393A
:1052A8000E94163A19F0E8E70E945339AE81EFE1FF
:1052B8000E94EA3D0E2EE5E20E94E53DE02161F004
:1052C800EDE60E944D37E8E50E9452370E949A3A6F
:1052D800DF01EE81EF51EC93AE81AE3231F4E9E3B8
:1052E8000E944D37E8E30E945237AE81AF3249F44D
:1052F800E8E70E944D37E5E00E945237E7E70E9451
:105308005737AE81A03331F4E0E30E94033AE0E579
:105318000E945737AE81A133B1F4E3E70E948F3A78
:10532800E8E70E945737A0910203A43160F0E4E552
:105338000E944E39EDE60E945339E0E30E94583945
:10534800EDE30E948239AE81A23341F4EEE30E947C
:105358004D37EBE00E945237E0E6E8AB0E94F039A7
:105368000E94FE3DE02111F00E949F3AAE81A333D6
:1053780029F40E94A53AE8E30E945737AE81A43386
:1053880089F4E8E70E944D37E8E30E9452370E940B
:105398009A3AA0912C03A083AD89BE89549711F441
:1053A8000E949F3AAE81A53349F4E8E30E944D3745
:1053B800E0E30E945237E4E50E945737AE81AC35EE
:1053C80049F4E7E70E944D37E9E30E945237E9E3E1
:1053D8000E945737AE81AD3509F086C0AFA5A83019
:1053E80008F044C0E7E70E94923A0E949A3AAFA5B3
:1053F800A083E7EAE0937A000E94D432E093510355
:10540800F0935203E7E2E0937A000E94A93AA83E9B
:10541800E3E0BE0740F00E949C38BF010E94A93A11
:105428000E943D38EC930E94A93AA436E0E0BE07FA
:1054380040F00E94A938BF010E94A93A0E9448384A
:10544800EC930E94A93A1A9750F00E945338BF0172
:105458000E94A93A0E9476360E945838EC930E941E
:10546800B438BF010E94A93A0E948C39AFA5A83070
:10547800E1F4E6E70E94103AE8E30E94AE3ADF0161
:10548800E0914703E1700E941F383E96DF01E091EA
:105498004703E695E1700E941F383F96DF01E091CF
:1054A8004703E695E695E170EC93AFA5A930E1F4E2
:1054B8000E94A53AE0E30E9457370E943A361A97AD
:1054C8004CF00E94A938BF010E943A360E94333737
:1054D8000E94F4370E945338BF010E943A360E9456
:1054E8006739E7E70E949939AE81AE3509F0BBC14B
:1054F800E0914903E030D1F40E94063AEBE00E94C3
:1055080057370E94FD36EA3048F00E945338BF01F1
:105518000E94FD360E94B03A0E94F4370E94B438C7
:10552800BF010E94FD36F0E00E94F437A0914903C4
:10553800A130F1F4E0E30E94B33AEBE00E94573760
:105548000E940237EA3048F00E94A938BF010E9441
:1055580002370E94B03A0E94F4370E945338BF01C4
:105568000E940237F0E00E94F437E7E70E94993979
:10557800A0914903A230F1F4E0E30E944D37E3E73C
:105588000E94B63A0E940737EA3048F00E94A938CC
:10559800BF010E9407370E94B03A0E94F4370E9468
:1055A8005338BF010E940737F0E00E94F437E7E75D
:1055B8000E949939A0914903A330E9F4EEE30E94CF
:1055C800B33AECE00E94AE3ABF010E940C37DF010B
:1055D8000E9462390E945338BF010E940C37DF01D4
:1055E8000E9433370E94F4370E94B438BF010E94EA
:1055F8000C370E94F437A0914903A430E9F4EEE394
:105608000E94B33AEBE00E94AE3ABF010E941A37FB
:10561800DF010E9462390E945338BF010E941A3785
:10562800DF010E9433370E94F4370E94B438BF016B
:105638000E941A370E94F437A0914903A530D1F58A
:10564800E3E70E944D37EBE00E9452370E9438375B
:10565800E83EA3E0FA0744F00E947738BF010E94B1
:105668003837DF010E945D390E943837E436A0E000
:10567800FA0744F00E949C38BF010E943837DF01C6
:105688000E9462390E9438373A9754F00E94A9382C
:10569800BF010E943837DF010E9433370E94F43778
:1056A8000E945338BF010E9438370E94F437EEE356
:1056B8000E949939A0914903A63059F5E8E70E945C
:1056C8004D37E0E00E94B63A0E941F37E436A0E06A
:1056D800FA0744F00E947738BF010E941F37DF01A4
:1056E8000E9462390E941F373A9754F00E949C38F2
:1056F800BF010E941F37DF010E9433370E94F43731
:105708000E94A938BF010E941F370E94F4370E94E7
:10571800B93AA0914903A73059F5E8E70E944D37F7
:10572800E1E00E94B63A0E942437E436A0E0FA0786
:1057380044F00E947738BF010E942437DF010E949D
:1057480062390E9424373A9754F00E949C38BF016E
:105758000E942437DF010E9433370E94F4370E94E9
:10576800A938BF010E9424370E94F4370E94B93A31
:10577800A0914903A83059F5E8E70E944D37E2E0C7
:105788000E94B63A0E942937E436A0E0FA0744F0AE
:105798000E947738BF010E942937DF010E946239D1
:1057A8000E9429373A9754F00E949C38BF010E9402
:1057B8002937DF010E9433370E94F4370E94A93845
:1057C800BF010E9429370E94F4370E94B93AA0917C
:1057D8004903A93009F047C0ECE70E948F3A0E94BC
:1057E8002331A031E7E2BE0738F00E946A380E94F0
:1057F80023310E94FA39EC930E942331A83EE3E05A
:10580800BE0740F00E947C38BF010E9423310E94ED
:105818003D38EC930E942331A436E0E0BE0740F007
:105828000E947738BF010E9423310E944838EC93C8
:105838000E9423311A9750F00E949C38BF010E94A1
:1058480023310E9476360E945838EC930E94A9387A
:10585800BF010E9423310E948C39E4E50E949439EB
:10586800E7E70E949939AE81AF3571F50E944E364F
:10587800AFE8B3E00E948631A091F603AA2342F470
:10588800E0918F03F09190030E94A03D0E94E337BE
:105898000E941538BF010E94E8370E9462390E94B1
:1058A800763A0E94E8370E9433370E94F4370E9404
:1058B8009A3ABF010E94E8370E946739EEE50E94D4
:1058C8004E39E1E00E945339AE81A03631F4E8E365
:1058D8000E94923AEDE00E945737AE81A13631F42A
:1058E800E8E70E94103AEEE30E945737AE81A236ED
:1058F80061F4E8E30E944D37FE01EE5BFF4F3696F8
:10590800A0913203A083E0E1E8ABAE81A33699F41D
:10591800E8E30E94923A0E949035EA17FB0718F4D0
:10592800ECE00E9457370E9490350E94973519F095
:10593800EBE00E94573731E0303108F089C00E940F
:10594800DE39EC91E03021F40E94DE39EFE3EC938C
:105958000E94DE39AC91A63021F40E94DE39EDE7D1
:10596800EC930E94DE39AC91A13021F40E94DE391B
:10597800E6E0EC930E94DE39AC91A23021F40E945B
:10598800DE39EBE5EC930E94DE39AC91A33021F4CB
:105998000E94DE39EFE4EC930E94DE39AC91A4302A
:1059A80021F40E94DE39E6E6EC930E94DE39AC91E0
:1059B800A53021F40E94DE39EDE6EC930E94DE3931
:1059C800AC91A73021F40E94DE39E7E0EC930E9405
:1059D800DE39AC91A83021F40E94DE39EFE7EC9370
:1059E8000E94DE39AC91A93021F40E94DE39EFE63D
:1059F800EC930E94DE39AC91AA3021F40E94DE3982
:105A0800E0E0EC930E94DE39AC91AB3021F40E94C7
:105A1800DE39E1E0EC930E94DE39AC91AC3021F440
:105A28000E94DE39E8E0EC930E94DE39AC91AD309B
:105A380021F40E94DE39E0E4EC930E94DE39AC9157
:105A4800AE3021F40E94DE39E9E0EC933F5F74CF79
:105A5800E0910103E695E6950E94BD3A0E94C33A9B
:105A68000E94C83A0E94C33A0E94D03A0E94C33AA0
:105A78000E94DB3A0E94C33A0E94A2390E94E23A8D
:105A88000E94E53A0E94E23A0E94EA3A0E94E23A0B
:105A98000E94EF3AEAABE0910103E695E695E695B8
:105AA8000E94BD3A0E94F53A0E94C83A0E94F53A0F
:105AB8000E94D03A0E94F53A0E94DB3A0E94FA3AD4
:105AC8000E94A2390E94FF3A0E94E53A0E94FF3ADA
:105AD8000E94EA3A0E94FF3A0E94EF3AEBABE0914B
:105AE8000103E6950E94BD3A0E94FA3A0E94C83A1C
:105AF8000E94FA3A0E94D03A0E94FA3A0E94DB3A8F
:105B08000E94F53A0E94A2390E94023B0E94E53A9F
:105B18000E94023B0E94EA3A0E94023B0E94EF3A2E
:105B2800ECABFE01E65BFF4FE0810E94BD3A0E94AC
:105B3800053B0E94C83A0E94053B0E94D03A0E9449
:105B4800053B0E94DB3AE52F0E94A239EA2BAE2FD3
:105B5800E52F0E94E53AEA2BAE2FE52F0E94EA3A9C
:105B6800EA2BAE2FE0910103E170EA2BEDAB0E9426
:105B78000A3B0E94BD3A0E940A3B0E940F3B0E94CA
:105B88000A3B0E94153B0E940A3B0E941E3B0E9452
:105B9800283B0E942C3B0E942F3B0E942C3B0E94DA
:105BA800363B0E942C3BE295E170EA2BEEAB0E945B
:105BB8003D3B0E94BD3A0E943D3B0E940F3B0E9424
:105BC8003D3B0E94153B0E943D3B0E941E3BE295D7
:105BD8000E94A2390E94423B0E942F3B0E94423BF6
:105BE8000E94363B0E94423BE295E170EA2BEFAB04
:105BF800E52F0E94493B0E943D3B0E94C83A0E9403
:105C08003D3B0E94D03A0E943D3B0E94DB3A0E94F5
:105C18004D3B0E94A2390E94523B0E94E53A0E94E5
:105C2800523B0E94EA3A0E94523B0E94EF3AE8AF88
:105C38000E94553B0E94BD3A0E94553B0E940F3B73
:105C48000E94553B0E94153B0E94553B0E941E3BFB
:105C58000E945A3B0E94A2390E94523B0E942F3B4D
:105C68000E94523B0E94363B0E94523BE295E170F3
:105C7800EA2BE9AF0E945F3B0E94BD3A0E945F3B5E
:105C88000E940F3B0E945F3B0E94153B0E945F3BB6
:105C98000E941E3BEE1FE0E0EE1F0E94A2390E9408
:105CA800643B0E942F3B0E94643B0E94363B0E944B
:105CB800643BE295E170EA2BEAAFE42FE2950E949B
:105CC800BD3A0E945F3B0E94C83A0E945F3B0E9417
:105CD800D03A0E945F3B0E94DB3A0E94053B0E943B
:105CE800A2390E946B3B0E94E53A0E946B3B0E94DE
:105CF800EA3A0E946B3B0E94EF3AEBAF0E946E3B80
:105D08000E94BD3A0E946E3B0E940F3B0E946E3B70
:105D18000E94153B0E946E3BE695E695E6950E942B
:105D2800733B0E2EA0E035FCA1E0EA2FEE0FEE0F3C
:105D3800EE0FE0290E94783BE2950E947E3B0E948C
:105D4800783B0E94363BEA2B0E94783BE295EF7045
:105D5800E695E170EA2BECAFFE01ED5BFF4FE081C9
:105D6800E695E695E6950E94BD3AFE01ED5BFF4F8C
:105D7800E081E695E6950E94833B0E94783B0E946D
:105D8800873B0E94783B0E94733BAE2FE42F0E9412
:105D9800283BEA2BAE2FE42F0E948E3BAE2FE42F38
:105DA8000E94913BE42FE695E170EA2BEDAFE42FDA
:105DB8000E94493B0E94963BE2950E94833BAE2F8E
:105DC8000E94963B0E94D03A0E94963B0E949B3BC1
:105DD800AE2F0E94963B0E94283BEA2BAE2F0E94D2
:105DE800963B0E948E3BAE2F0E94963BE6950E9402
:105DF800913B0E94963BE170EA2BEEAFE42F0E94A4
:105E08005A3B0E94BD3AE8A90E94833BAE2FE8A9FD
:105E18000E94873BAE2FE8A9E695E6950E94733B62
:105E2800AE2FE0910103E2950E94A239EA2BAE2F32
:105E3800E42FEE1FE0E0EE1F0E947E3BAE2FE8A9A4
:105E4800E695E695E6950E94913BE8A9E295E17012
:105E5800EA2BEFAFFE01F1963F960F01E8A90E94E9
:105E6800493B0E949F3BE2950E94833BAE2F0E94D4
:105E78009F3B0E94D03A0E949F3B0E949B3B0E94FE
:105E8800A43B0E94283BEA2B0E94A43B0E948E3B25
:105E98000E94A43BE6950E94913B0E94AA3BE170B8
:105EA800EA2BD001EC93FE01F19670960F01E8A958
:105EB8000E945A3B0E94BD3A0E94AA3BE2950E946A
:105EC800833B0E94A43B0E94D03A0E94AA3B0E94B6
:105ED8009B3BAE2F0E949F3B0E94283BEA2BAE2F94
:105EE8000E949F3B0E948E3BAE2F0E949F3BE695EF
:105EF8000E94913B0E949F3BE170EA2BD001EC93FA
:105F080033FE0DC031E0313150F4E32FF0E0DE0113
:105F1800D196AE0FBF1FEFEFEC933F5FF4CF0E9417
:105F2800AF3B3D3078F40E94B53BA2E5B8E00E9453
:105F3800B43DE17011F45D9801C05D9A0E94BC3BCC
:105F48003F5FEFCF0E94C43B3D3078F40E94B53BE1
:105F5800A0E3B8E00E94B43DE17011F45D9801C07F
:105F68005D9A0E94BC3B3F5FEFCF0E94C43B3D302F
:105F780078F40E94B53BA2E0B8E00E94B43DE1701D
:105F880011F45D9801C05D9A0E94BC3B3F5FEFCF62
:105F98000E94C43B3D3078F40E94B53BA6E0B8E0CF
:105FA8000E94B43DE17011F45D9801C05D9A0E94B1
:105FB800BC3B3F5FEFCF0E94C43B3D3058F50E9489
:105FC800CD3BA0913F030E947533A0913E030E94F0
:105FD800BD34A0E0F099A1E00E94393461F0ECE012
:105FE800E31BA2E1B8E00E94B43DE17011F45D98B2
:105FF80001C05D9A0BC0ECE0E31BA0E1B8E00E9491
:10600800B43DE17011F45D9801C05D9A0E94BC3BFB
:106018003F5FD3CFA0913F030E947533A0913E0309
:106028000E94BD34A0E0F099A1E00E94393419F033
:10603800E1E0E0933E03E0913F03E03019F4E0E053
:10604800E0933E035D9A84E08A95F1F7289A84E00C
:106058008A95F1F7289884E08A95F1F731E03A308B
:1060680088F40E94CD3BE9E0E31BA0E4B1E00E9484
:10607800B43DE17011F45D9801C05D9A0E94BC3B8B
:106088003F5FEDCF21E02131D8F431E03930B0F471
:106098000E94CD3BE22FF0E0DE01D196AE0FBF1F8C
:1060A800AC91E8E0E31B0E94AC3DE17011F45D980F
:1060B80001C05D9A0E94BC3B3F5FE8CF2F5FE3CFF2
:1060C8005D9A85E28A95F1F7289A84E191E0019733
:1060D800F1F70E946633A92D0E94D23BAB2D0E9496
:1060E800D23BAA2D0E94D23B0E948F360E2A0E94D4
:1060F800E034E0E0F0E060E07FEB0E948A3D0E2AA9
:106108000E9438350E2A0E942F34E02929F0E0E059
:10611800E0936B03E0936C03F09B03C0E0E0E09333
:106128003F03A82DE4E60E94F93D0E2EA0E0F09969
:10613800A1E00E942C3329F00E94D032F09AE89412
:1061480033F80C948406FFCFAA93E091C000E07264
:10615800E1F3E881E093C60021960895A0915503E4
:10616800B09156030895A091C703B091C8038091D8
:10617800C9039091CA030895E0E0F0E061EE75E488
:106188000E94253D0895E0916103F091620308950E
:10619800662777270E944D3C0E94103F0895E091A2
:1061A8006D03F0916E030895A091CF03B091D003D1
:1061B8008091D1039091D2030895E0E0F0E060E28D
:1061C80071E40895A0916103B09162030895E0E03D
:1061D800F0E00E94223E0895A0916D03B0916E03F5
:1061E8000895E091F703F091F8036091F903709135
:1061F800FA0308950E94143CED93FC930895A0912E
:10620800E303B091E4038091E5039091E6030895D8
:10621800E0E0F0E06AE774E40E94D73CDF01CB01DC
:10622800ABCFA091DF03B091E0038091E10390919F
:10623800E2030895E0E0F0E060E070E00895A091E6
:106248007503B091760308950E94243F0E94803C14
:106258000895A0910704B0910804809109049091D1
:106268000A040895E0917B03F0917C0360917D031B
:1062780070917E030895A4E6B0E080E090E00E946B
:10628800503EDF01CB01E091DF03F091E003609124
:10629800E1037091E2030E941F3F0895E0917303A8
:1062A800F09174030895E0937303F09374030895D1
:1062B800A091FF03B0910004809101049091020421
:1062C8000895E093FF03F093000460930104709332
:1062D80002040895A0917B03B0917C0380917D0313
:1062E80090917E0308950E94503EDF01CB01E0911A
:1062F800FF03F091000460910104709102040E9470
:106308001F3FA2CF0E94163CED93FC930895E0E056
:10631800F0E061EE75E40E94D73C0895A091E70390
:10632800B091E8038091E9039091EA030895E0E0D1
:10633800F0EC69E774EC0E946A3D0895E7EEF3E03B
:10634800E0939103F09392030895E091E703F091AD
:10635800E8036091E9037091EA030895E091EB0383
:10636800F091EC036091ED037091EE030895A09114
:10637800CB03B091CC038091CD039091CE030895C7
:10638800E093CB03F093CC036093CD037093CE03DB
:106398000895A091D303B091D4038091D50390912F
:1063A800D6030895E091CB03F091CC036091CD031F
:1063B8007091CE030895A091DB03B091DC03809126
:1063C800DD039091DE030895E0917703F09178035F
:1063D8006091790370917A030895E0937703F093BD
:1063E80078036093790370937A030895EDDFAFE53E
:1063F800B0E00E94453F0895A0917703B0917803DB
:106408008091790390917A030895D7DE0E94D73C52
:106418000895E0E00E94F93D0E2E0895A091AB0387
:10642800B091AC038091AD039091AE0308950E2214
:10643800A0912703ECE30E94F43D0895A0916B031B
:10644800B0916C030895A0916903B0916A03BFCE1F
:10645800E0916903F0916A030895A4E6B0E00C9412
:10646800D73BE7EAE0937A00A4E00C94CA03EF2F45
:10647800F0E06E2EE7E2E0937A000895E7EAE09311
:106488007A00A3E00E94CA03EF2FF0E09E2EE7E215
:10649800E0937A000895E7EAE0937A00A1E00E9489
:1064A800CA03EF2FF0E0BE2EE7E2E0937A000895EA
:1064B800E0E0F0E00E944D3F0895EBE0E093100427
:1064C800E8EBE09311040895E0938103F0938203CD
:1064D8000895E0938303F09384030895E0935903A8
:1064E800F0935A0308950E94CC3D0E944D3C0E94AF
:1064F800103F089562DE0E94253D0895E0935F03F2
:10650800F09360030895E0937B03F0937C0360931A
:106518007D0370937E030895E0936903F0936A0303
:106528000895ADE5B0E00E94353F0895E0936F030C
:10653800F09370030895E0933903E0E0E0932404B6
:106548000895E0910F04F0E0E0939903F0939A0323
:10655800E0911004F0E0EADFE0911104ECCFE0E014
:10656800E0930B04E0930C04E0930D04E0930E0415
:10657800E0930F04A2CFE0E0E0931204E093130449
:10658800E0931404E0931504E09324040895E09341
:106598009903F0939A030895AAE0B0E00C94D73BCE
:1065A8000E94CA030E94C13D0E94BD3D0895E7EACA
:1065B800E0937A00A0E00E94CA03EF2FF0E008956C
:1065C800E093AF03F093B0036093B1037093B20309
:1065D8000895E0915903F0915A030895E091AF03AB
:1065E800F091B0036091B1037091B2030895E7E2AE
:1065F800E0937A008AE48A95F1F708958AE48A9507
:10660800F1F7E7EAE0937A000895A7E00E94CA0349
:10661800EF2FF0E0E0934F03F09350030895A0911B
:106628004F03B09150030895E2E3F0E00E94223E48
:106638000E2E0895A98DBA8DF7CFEEE1F0E00E94F5
:106648001C3E0E2EA52DE1E00E94F93D0E22089574
:10665800E0E00E94D63DE0210895EAEFF0E00E94D4
:10666800223E0E2EA52DE1E00E94F93D0E2208954E
:10667800E4E00E94F43DE0210895E0934F03F09395
:1066880050030895E0E0E0934F03E093500308952A
:10669800E4E00E94D63D0E2E0895A9A1E5E00E94EF
:1066A800D63D0895AA2DEAE00E94F43D0E2E0895E5
:1066B800A0E0F3FCA1E0E0E00E94D63D0E22A02F6E
:1066C800E3E60895A62DEAE00E94F43D0E2E089513
:1066D800A5DEE2E0F0E060E070E00E94383EE021F4
:1066E8000895E1E00E94D63D0E2E0895A09114036E
:1066F800AFCFE3E00E94D63D0E2E0895E0914F0300
:10670800F09150030895F297ADE7B0E00E94483E3B
:106718000F010895F0E0DE019796AE0FBF1FEC91D0
:10672800F0E0D0010E94803EA8DF79DFA93CE0E0DC
:10673800BE070895EB85FC8572DF0E94483EDF01A5
:10674800E4E1F0E00E94803E98CFF0E0DE019B9605
:10675800AE0FBF1FEC91F0E062DF0E94483EDF0100
:10676800E4E6F0E00E94803E88CFE12FF0E0DE0111
:106778009396AE0FBF1F0895A091A303B091A403F1
:106788008091A5039091A6030895E8EEF3E060E0F8
:1067980070E00E94BD3EDF01CB01B0DF662777279E
:1067A8000895EC91F0E0A0E4BCE90E94803EE4DFAB
:1067B800662777270895E093A303F093A4036093D3
:1067C800A5037093A6030895D7DFDFCF0E949B3DF2
:1067D800E5E0F0E060E070E00E94403E08950E942D
:1067E8009B3DE4E1F0E060E070E00E94383E0895EF
:1067F8000E949B3DA431E0E0BE07E0E08E07E0E0A8
:106808009E070895E091AB03F091AC036091AD034E
:106818007091AE03A0E5B4E180E090E00E947B3E79
:10682800CACFE8EEF3E060E070E00895A02FE3E659
:106838000E94F43D0895A0E0F0FCA1E009CFEFDE4E
:10684800E0E0F0E00E94FE3D0895E89425F8E0E0DD
:10685800E09329030895E3DEBACC0E22A0E022FCDF
:10686800A1E0E1E00E94D63D0895E1E00E94D63D16
:10687800E0210895A0E025FCA1E033CFAF8DE3E04F
:106888000E94DB3DE0210895E0933603DECF0E2E13
:10689800A98DBA8DE0E0F0E00E94FE3D0E22089539
:1068A800A0E021FCA1E0E0E00E94D63D0895E0913F
:1068B8000403F0E03597B3DE0E941C3E0E2EE091F3
:1068C8003503ACDDFF27662777270895A0E022FC73
:1068D800A1E0BECEEB89FC89A091AF03B091B003D3
:1068E8008091B1039091B203662777270E94383EC2
:1068F8000E2EEAE0F0E060E070E00E94403E08956D
:106908006DDEAB89BC89882799270E949B3D089535
:10691800A630E0E0BE07E0E08E07E0E09E070895BD
:10692800A0918103B09182030895E0918103F091D1
:1069380082030895EB89FC89A091AF03B091B0035D
:106948008091B1039091B203662777270895EB856C
:10695800FC85A091F303B091F4038091F503909125
:10696800F603662777270E944D3C0E94903D0E2E25
:106978000895E0E00E94D63D0E22089550DEEAE038
:106988000E94703E0895EB85FC85A091F303B091B9
:10699800F4038091F5039091F603662777270E9408
:1069A8004D3C52CCA0918303B09184030895E091AB
:1069B8008303F09184030895A091F303B091F40345
:1069C8008091F5039091F6030895662777270E9432
:1069D8004D3C0895E091F303F091F4036091F503C1
:1069E8007091F603AB85BC85882799270E94213FC3
:1069F8002BCC0E94CC3D0E944D3C0895EAE0F0E08B
:106A08000E94933E3ACEE091180308DDFF276627DF
:106A180077270895E0938B03F0938C030895E09112
:106A28001803F0E0FBDC0E94CC3D0E949B3D0895DA
:106A38000E94763EA0918B03B0918C030895E0915B
:106A48008B03F0918C030895A0911803BB27E09164
:106A5800AB03F091AC036091AD037091AE030E945B
:106A6800D13D0E949B3D0895A98DBA8DB0CBA0E081
:106A7800F099A1E0E1E00E94D63DD9CC0E22A02FEA
:106A8800E3E60E94D63DE02108950E2EA09127034B
:106A9800ECE30E94F43D0E2208950E944D3FA1E0D0
:106AA800B0E00C94D73BE091DF03F091E0036091F4
:106AB800E1037091E203A1E4B0E00E94163CEDCF3F
:106AC800A9E4B0E00E94163CE8CFE8DBABE4B0E014
:106AD800E4CF0E94553FA1E0B0E00C94D73BE09191
:106AE8007503F0917603ADE5B0E00E944D3F08953F
:106AF800EAE00E94F93D0E2E0895AB2DEAE00E94CF
:106B0800F43D0E2EA0E027FCA1E033CFE091320344
:106B1800F0E0E05EFC4F0895ED85FE850E94C13DE2
:106B2800A62DB0E008950E94163E0E2EA62DEAE08E
:106B38000E94F93DE0210895A92DEAE00E94F43D64
:106B48000E2E0895E0910D03F0E0E85FFC4F0895E4
:106B5800E0915F03F09160030895A02FE3E60E949F
:106B6800D63DE0210895E0913B03EF5FE0933B03BE
:106B7800E0913A03A0913B03EA170895E0931903C3
:106B8800F0E037DFACE5BFE882E290E40E94D73C52
:106B9800A3ECB5EF88E490E40E94D73CAFE5B3E0FE
:106BA80029CB0E941C3E0E2EA0E023FCA1E00895F4
:106BB800A0915F03B09160030895A0DCC9DF05DFF1
:106BC800DF01CB01ECE5FFE862E270E40E94253DBD
:106BD800DF01CB01E3ECF5EF68E470E40E94253DAA
:106BE800A9E1B3E00E94143CEC930895A0917303CB
:106BF800B09174030895E0912C03F0E0E65BFC4F3C
:106C0800A0810895A0912C03B0E0A65BBC4FEC9145
:106C18000895A0913203B0E0A05EBC4FEC910895B6
:106C2800AE81E3E60E94D63D0E2E76CFE1E00E94CB
:106C38002D3FEA1B0E94803F0895E0919903F0914F
:106C48009A03A3EFB3E04FCCE093F303F093F4037C
:106C58006093F5037093F6030895E091F303F091C0
:106C6800F4036091F5037091F6030895A0919F03D2
:106C7800B091A0030895F1DFA0E0B0E080E09FE3C9
:106C88000895E093E303F093E4036093E5037093BE
:106C9800E603089591DEB9CBE0DFAFE8B3E032CB8D
:106CA800EA1BFB0BA6DEDF01CB01EAE9F9E969E2A1
:106CB80071E40E94253DDF01CB01E0E0F0E068E5EA
:106CC80071E4C2CAEE0FFF1FA0E0B4E00E942A3FA1
:106CD800E7CFE091C303F091C4036091C5037091BD
:106CE800C6030895EAE0F0E00E94803E0895A0916E
:106CF800C303B091C4038091C5039091C60308955E
:106D0800B1DAB9CAE093BF03F093C0036093C1033B
:106D18007093C203089582DB8DDA0E94403E089585
:106D2800EF85F889A091AF03B091B0038091B103CA
:106D38009091B203662777270895A091AF03B09189
:106D4800B0038091B1039091B2030895EA0FFB1F3D
:106D5800E0935D03F0935E0308950E94A830A0912C
:106D68004F030C94A8300E94A830E0915E03AE2F28
:106D78000E94A830A0915D030C94A830F0E0AE0FFB
:106D8800BF1FE0911B03F0E00895F0E0AE0FBF1FB6
:106D9800E0914103F0E0AE0FBF1FE0914203089578
:106DA8000E94A830A09116030E94A830A091170352
:106DB8000C94A8300E94A830A0911B030C94A83012
:106DC8000E94A830A0911C030C94A830A1E00E9456
:106DD800A830A6E30C94A8300E94A830A0915D03C7
:106DE8000C94A8300E94A830A0E00E94A830A0E02F
:106DF8000895A6E3B0E00E94393F0895A7E3B0E004
:106E08000E94393F0895A8E3B0E00E94393F0895F1
:106E1800A1E5B0E00E94353F0895A091B303B09179
:106E2800B4038091B5039091B6030895A3E5B0E04B
:106E38000E94353F0895A7E5B0E00E94353F0895C8
:106E4800A9E5B0E00E94353F0895ABE5B0E00E94A7
:106E5800353F0895A091A103B091A2030895EAE0F7
:106E6800F0E00E94933E0895A5E5B0E00E94353F0A
:106E78000895DE01AD5BBF4FEC930895EAE0DE01B3
:106E8800AB5BBF4FEC930895DE01AA5BBF4FEC9359
:106E98000895DE01A95BBF4FEC930895DE01A85B5E
:106EA800BF4FEC930895DE01A75BBF4FEC930895A5
:106EB800EAE0DE01A65BBF4FEC93DE01A55BBF4FA6
:106EC800EC93DE01A45BBF4FEC93DE01A35BBF4FE5
:106ED800EC93DE01A25BBF4FEC93DE01A15BBF4FD9
:106EE800EC93DE01A05BBF4FEC93DE01AF5ABF4FBE
:106EF800EC93089559E0E0913803E170EE0FAE2F5E
:106F0800E0913803E695E170EE0FEE0FEE0FEA0F11
:106F18000E2E0895E0913803E695E695E170AE2FC0
:106F2800E0E0F5FCE1E0EA2BEE0FEE0FE00D4E2F6E
:106F380008955E2FE0913803E170EE0FAE2FE091D7
:106F48003803E695E170EE0FEE0FEE0FEA0F0E2E06
:106F5800E1CFE295E07FEE0FEE0F0895E0E020FC30
:106F6800E1E0E093010359CFAA30E0E0BE07E0E09A
:106F78008E07E0E09E07089551DAEAE0F0E060E06D
:106F880070E008950E94BD3EDF01CB01EAE0F0E029
:106F980060E070E00E94D73E0895FE01EE5BFF4F6F
:106FA80034960895DE01AB5BBF4FEC930895E091F2
:106FB8008D03F0918E030E94A03DDF0150CFE09336
:106FC8008F03F09390030895A0918F03B0919003DD
:106FD8000895FE01EE5BFF4F3196BF01F5DF3FCF0D
:106FE800DF01EAE0F0E00E94C53EDB01EC93089582
:106FF800FE01EE5BFF4F3296BF01E6DFEAE0F0E00C
:107008000E94C53EDB01EC930895E0912C03A3E9AF
:10701800B3E0F0E0EE0FFF1FAE0FBF1F0E940C3F62
:107028000895FE01EE5BFF4F35960895E4E6F0E023
:1070380060E070E00895EC93FE01EE5BFF4F089569
:10704800ECDEEAE0F0E060E070E00895A0E020FC0B
:10705800A1E0EA2FE295E07F4E0F0895A091570333
:10706800B09158030895FE01EE5BFF4F3D96BF01B6
:10707800F5CFE8EEF3E00E94803EDF01EAE0F0E0C1
:107088000E94C23EDB010895E4E6F0E00E94803EE3
:10709800DF01EAE0F0E00E94C23EDB010895FE0154
:1070A800EE5BFF4F3E960895DF01EAE0F0E00E94B4
:1070B800C23EDB0108950E94C23EDB01EC930895B5
:1070C800E2E0DE01A65BBF4FEC930895FE01EE5BA4
:1070D800FF4F3996BF010895BB27EAE0F0E00E9410
:1070E800C53EDB010895FE01EE5BFF4F3B96089518
:1070F800FE01EE5BFF4F3A9608950E94983EDF012D
:10710800CB01EAE0F0E060E070E00E94D33E089531
:10711800A031E7E2BE07E0E08E07E0E09E070895B1
:10712800A83EE3E0BE07E0E08E07E0E09E07089592
:10713800FE01EE5BFF4F3C960895A436E0E0BE07E3
:10714800E0E08E07E0E09E070895FE01EE5BFF4F4A
:107158003D96089551D9EAE0F0E060E070E00895C6
:10716800FE01EE5BFF4F3F960895DE01A55BBF4F22
:10717800EC93E4E7DE01A45BBF4FEC930895E0E4F1
:10718800DE01A05BBF4FEC930895DF01CB01E0E087
:10719800F0E060E171EC0E946A3D0895E0E4DE01F0
:1071A800A15BBF4FEC930895DF01CB01E0E0F0E075
:1071B80066EC72EC0E946A3D0895E0E4DE01A25B91
:1071C800BF4FEC930895DF01CB01B1C8E0E4DE01C5
:1071D800A35BBF4FEC930895A091B703B091B80398
:1071E8008091B9039091BA030895F6DFEAE0F0E0E0
:1071F80060E070E00895E0918903F0918A030E94AD
:10720800A03DE0938903F0938A0308952BD8A4E660
:10721800B0E080E090E067C8A0918903B0918A034C
:107228000895BF01F9DFE0E1F7E20E94933ED8CE6E
:10723800BF01F2DFE8EEF3E00E94933ED1CEBF013A
:10724800EBDFE4E6F0E00E94933ECACEBF01E4DF44
:10725800EAE0F0E00E94C53EDB01EC930895E0E52A
:10726800DE01A35BBF4FEC930895A0919103B09109
:1072780092030895BF01F9DFE4E6F0E00E94933E2F
:10728800AFCEBF01F2DFEAE0F0E00E94C53EDB01CD
:10729800EC930895DE01A55BBF4FEC930895DE01E2
:1072A800A45BBF4FEC930895DE01A35BBF4FEC9343
:1072B8000895E8EEF3E00E94933E92CEE4E6F0E013
:1072C8000E94933E8DCEEAE0F0E00E94C53EDB01CD
:1072D800EC930895E98DFA8DF695E7950895E8EC15
:1072E800F0E00E94803EE0CEE4E1F0E00E94803EC3
:1072F800DBCEE989FA89F695E7950895DE01A25B68
:10730800BF4FEC930895A0916303B091640308956F
:10731800EAE0F0E0D0CEDE01A15BBF4FEC93089528
:10732800DE01A05BBF4FEC930895DE01AF5ABF4F5B
:10733800EC9308950E940A3E0E2E8CCDE170EE0F5C
:10734800EE0FEE0F0895ECE7AADF89CFA9A1E4E0DC
:107358000E94D63DAE2FE0E020FCE1E0EA2308954C
:10736800AE2FE0E020FCE1E0EA230895ECE7D3DF6C
:10737800E0E5D6CFE7E7CFDFE9E3D2CFF0E00E9440
:10738800103EEECFE4E10E94F93DE0210895E0933C
:107398002C03E8E77FCF83DFEAE086DFE9E7AEDFAB
:1073A800E0E5B9DFE0E5BCDFEAE0BFDFE1E0E0937C
:1073B8003F030895E32FF0E0DE01AE5BBF4FAE0F51
:1073C800BF1F08950E94D63D0E2EAE8108950E94DB
:1073D800D63D0E2AAE810895AE81E2E30E94D63DE5
:1073E8000E2EAD89BE89E4EAF1E00895E0E1F7E206
:1073F8000E94803E59CEBF01AD89BE8973CC49DD5C
:10740800E9E74CCDEDE645DDE3E748CDE9E341DDCD
:10741800E0E544DDEEE347CD3CDDE7E73FCDAE8177
:10742800E5E0D0CFE3E10E94D63DE0290895E72DBD
:10743800F0E0DE019396AE0FBF1F0895A091A70359
:10744800B091A8038091A9039091AA030895EC91A3
:10745800F0E0A0E4BCE90E94803EF0DF66277727D1
:107468000895E093A703F093A8036093A90370938A
:10747800AA030895E3DF89C9E091AB03F091AC0357
:107488006091AD037091AE03A0E5B4E180E090E0B7
:107498000E947B3EE6CF51DCEAE0F0E060E070E07D
:1074A80008952CD9F695E795E8C8E8ABB8D8A4367E
:1074B800E0E0BE070895BF01B2D8E6CDFE01EE5B5D
:1074C800FF4F3696BF01ABD80DCCFE01EE5BFF4FE8
:1074D8003796BF01A4D81CCF0E94D63D0E2EA0918E
:1074E8004203C3C9FE01EE5BFF4F3696BF01089504
:1074F800BF01A0917103B09172030895A0915B033D
:10750800B0915C030895E8E5C4DCE4E5C7CCEDE69A
:10751800C0DCE8E3C3CCBDDCE0E5C0CCBADCEEE51A
:10752800BDCCA0916703B09168030895FE01EE5B9E
:10753800FF4F37960895E0E0EEDEE1E7F1DEE1E7A0
:10754800F4CEE3E7A6DCE4E7A9CCA0915103B0911F
:1075580052030895A8DCF9CDF0E0DF0180CC99DC76
:10756800ECE79CCC9BDCEBE09ECCE3E6D9DEE9E3E0
:10757800DCCEE170E795E0E0E795AE2F0895FE01D7
:10758800E95BFF4FE0810895E295EF70E695E170C1
:10759800E0DCEA2BAE2F0895E295EF70E695E695CC
:1075A800E170E295E07FEE0FEA2BAE2F0895E295A9
:1075B800E170E295E07FEA2BAE2F0895EA2BAE2F1B
:1075C800DECFE695E170EE0FEE0F0895E695E695AD
:1075D800E170EE0F0895E695E695E695E170EA2BE1
:1075E8000895FE01E85BFF4FE0810895FE01E75B27
:1075F800FF4FE0810895EA2BAE2FF8CFEA2BAE2F8C
:10760800F0CFFE01E55BFF4FE0810895FE01E15BED
:10761800FF4FE0810895E695E1709BDCEA2BAE2FE1
:107628000895E695E695E170E295E07FEE0FEA2B86
:10763800AE2F0895E695E695E695E170E295E07F30
:10764800EA2BAE2FE52F0895E695E695E69576CEDA
:10765800EA2BAE2FDBCFE295EF70E695E170EE0FE7
:10766800EE0F0895E295EF70E695E695E170EE0F5E
:107678000895FE01E25BFF4FE0810895EA2BAE2FEB
:10768800FE01E05BFF4FE0810895E295EF70E6951B
:1076980070CFFE01E35BFF4FE0810895EA2BAE2F28
:1076A800F8CFFE01E05BFF4FE0810895E295EF70AF
:1076B800E695E6950895FE01E45BFF4FE0810895A5
:1076C800EA2BAE2FFE01EF5AFF4FE0810895EA2B17
:1076D800AE2F97CFFE01EF5AFF4FE0810895E1707A
:1076E800E295E07FEA2B0895AE2FFE01ED5BFF4F98
:1076F800E0810895E170EE0FEE0FEA2B0895E17036
:1077080028DCEA2B0895E695E170E295E07FEE0F1C
:10771800EA2B0895E695E695EDCFE170EE0FEA2B9A
:10772800AE2F0895FE01EC5BFF4FE0810895E295CE
:10773800EF70E695D4CFFE01EB5BFF4FE081089533
:10774800AE2FFE01EA5BFF4FE0810895FE01EA5B80
:10775800FF4FE0810895289885E28A95F1F731E096
:1077680008955E9884E08A95F1F7ECE0E31B0895AC
:1077780084E08A95F1F75E9A84E08A95F1F7089596
:107788005D9A85E28A95F1F7289A85E28A95F1F75C
:10779800E2CF5E9884E08A95F1F70895EAE00E94C6
:1077A800F43D0E2A0895109639F08DEC9AE0019771
:1077B800F1F7A8951197C9F7089530976040704080
:1077C80009F070580895552342F4503811F4E0FF39
:1077D80004C03196691F791F6BF050E8572711F4E0
:1077E8005F93CFC05F3F31F0660F000C57956795E8
:1077F800752F08955F9300200AF0CFC0C8C050E8E5
:10780800192E1522880F991F9527550F879550E82F
:10781800072E0522660F771F7527550F6795089560
:10782800689401C0E8945F93F2DF703818F07F3FE6
:1078380008F4A7C056E1571BAAF4519558300EF426
:10784800593030F0EFEFFFEF6FEF7FE777F91AC0AD
:1078580077275523B9F0EE0FFF1F661F771F5A953C
:10786800D1F710C07727583028F0EF2FF62F672F61
:107878005850F9CF552331F076956795F795E795E8
:107888005A95D1F700200AF45BD15F910895689466
:1078980001C0E894309760407040B1F0002426F0B1
:1078A800772312F400944CD1172E7EE1112032F088
:1078B8007A95EE0FFF1F661F111CF9CFEF2FF62FD9
:1078C800612D5F938ADF5F9108954F93AF01FD01AA
:1078D800DA01AB01BC01CA01402D012C142E4F91D5
:1078E8000895EA0FFB1F681F0895E095F0956095CD
:1078F800EF5FFF4F6F4F08955F9381DF903871F10D
:1079080050E8152604C05F937ADF903839F1703853
:1079180021F1572F591B2BF112F4D7DFFACF583129
:1079280018F0AA27BB278827583028F0AB2FB82F84
:1079380088275850F9CF552329F08695B795A795EC
:107948005A95D9F7502D512572F0CBDF38F4679549
:10795800F795E795739513F420C0B7DF3EDF5F9185
:107968000895D8F7FBCFEA1BFB0B680B51F010F416
:107978000094BBDF662392F3EE0FFF1F661F7A9514
:10798800CBF7EE27FF27662777275F910895EFEF5C
:10799800FFEF6FE77FEF5F910895EFEFFFEF6FE77E
:1079A8007FE75F9108955F932ADF703851F390382D
:1079B80041F301240894791F23F41CF300203AF3BF
:1079C800ECCF0F921F932F933F934F9311272227AA
:1079D8009927689FA0018F9F302D410D591F6B9FDC
:1079E800300D411D591F8E9F27D0BF9F25D06A9FFC
:1079F80023D0BE9F1DD0AF9F1BD0AE9F110D291F56
:107A0800391F491F591FE32FF42F652F522F4F910C
:107A18003F912F911F910F9066232AF0550FEE1F6B
:107A2800FF1F661F02C073954BF2CDDE5F9108956C
:107A3800100D211D391F02C0200D311D491F591F6E
:107A480008955F93DCDE703821F411200AF49FCF8B
:107A5800A4CF903809F495CF01240894970B1BF410
:107A6800D4F30020F3CF792F1F932F933F934F9395
:107A780011241127222733274427552790E2AE17D0
:107A8800BF078607410730F0AE1BBF0B860B410BC3
:107A9800089401C08894551F221F331F111CAA1F68
:107AA800BB1F881F441F9A9551F7F901612D4F910B
:107AB8003F912F911F91662332F0550FEE1FFF1F44
:107AC800661F7A9543F27FDE5F91089599239AF0B5
:107AD800772342F0971748F029F4AE17BF078607B7
:107AE80020F031F098948894089598940894089513
:107AF8001894889408957723C2F7971798F3A9F7ED
:107B0800EA17FB07680788F399F3ECCFDFDFE1E0BA
:107B180009F008F0EE270895D9DFE1E009F008F44C
:107B2800EE270895EA0FFB1F681F791F0895AE1B03
:107B3800BF0B860B970B0895F195E195F0400895DA
:107B4800F09560957095E195FF4F6F4F7F4F0895C1
:107B5800EE230E2EEA2F19F0E6950A94E9F7089518
:107B6800EE230E2EFD0121F0F695E7950A94E1F734
:107B78000895F695E795F695E795F695E795F695C0
:107B8800E7950895FE2FFF0FFF0B6F2F7F2F0895A6
:107B98006F2F660F660B762F08958B2F880F880B33
:107BA800982F0895EA17E1E009F0EE270895EA17FB
:107BB800E1E009F4EE270895AE17E1E00CF4EE27B2
:107BC8000895AE17E1E00CF0EE270895EA17E1E01A
:107BD8000CF0EE270895AE17E1E008F4EE270895BB
:107BE800AE17E1E008F0EE270895EA17E1E008F0A3
:107BF800EE270895EA17FB07E1E009F0EE2708955C
:107C0800EA17FB07E1E009F4EE270895AE17BF076E
:107C1800E1E00CF0EE270895EA17FB07E1E00CF02D
:107C2800EE270895EA17FB07E1E008F4EE27089528
:107C3800AE17BF07E1E008F0EE270895EA17FB0743
:107C4800E1E008F0EE270895EA17FB0768077907CF
:107C5800E1E009F0EE270895EA17FB0768077907BE
:107C6800E1E00CF4EE270895AE17BF0786079707E3
:107C7800E1E00CF0EE270895EA17FB07680779079B
:107C8800E1E00CF0EE270895FA9FF02DEB9FF00D40
:107C9800EA9FE02DF10D08957A9F702D6B9F700D6E
:107CA800F89F700DE99F700D6A9F602D710DFB9F05
:107CB800600D711DE89F600D711D8827FA9FF02DDA
:107CC800610D781FEB9FF00D611D781FEA9FE02D75
:107CD800F10D681F781F08956E2F6A9FF0016B9F42
:107CE800F00D089574D0D0DF0EF426DF08957DD00E
:107CF800D3DF0EF425DF08950024112490E1AA0FA4
:107D0800BB1F001C111C0E1A1F0A18F40E0E1F1E92
:107D180001C0A1609A9599F7FD01D001089557D047
:107D2800EBDF0EF409DF08953F934F935F93002430
:107D380011244427552730E2AA0FBB1F881F991F1B
:107D4800001C111C441F551F0E1A1F0A460B570B07
:107D580028F40E0E1F1E461F571F01C0A1603A953A
:107D680059F7FD01BC01D001CA015F914F913F91C4
:107D780008953BD0D9DF0EF4E3DE0895BDDFFD01A1
:107D88000895E894B7FF04C0A095B095119668943B
:107D9800F7FDD2DEB1DFFD010EF4CEDE0895C4DFBB
:107DA800FD01BC010895E89497FF09C0A095B0951E
:107DB80080959095AF5FBF4F8F4F9F4F689477FD29
:107DC800BFDEB2DFFD01BC010EF4BADE0895E8940F
:107DD800F7FF02C0B1DE6894B7FF06C0A095B09562
:107DE800119600F8039400FA0895E89477FF02C00A
:107DF800A7DE689497FF0BC00024A095B0958095E6
:107E080090951196801D901D00F8039400FA08952E
:107E1800ED91FC9111970895ED93FD936D937C93EB
:107E28000895A881B9818A819B810895E883F9839F
:107E38006A837B830895689401C0E89401D02ADDA1
:107E4800182E862F612D192E972F712D1B2EBF2FBF
:107E5800F12D1A2EAE2FE12D0895129602D0BF01F2
:107E68001297119602D0FE2F1197F999FECFFF9322
:107E7800FFB7F894A1BDB2BDF89AE0B5FFBFFF9176
:107E8800089507D012960F01FB0103D0F001129755
:107E9800089507D01196EF93EF2F03D0EF91119724
:107EA8000895F99B02C0A895FCCF9FB7F894A1BD8F
:107EB800B2BDF89A80B5E81719F0E0BDFA9AF99AB8
:107EC8009FBF089500240E160F060606070608959C
:107ED80000240A160B06089500240A160B06080645
:107EE80009060895EA17FB07680779070895AE178A
:107EF800BF07860797070895E894EE2309F068946A
:107F08000895AC0FBD1F05900D928A95E1F708956D
:00000001FF
